:100000007AC70000A9C70000A7C70000A5C7000065
:10001000A3C70000A1C700009FC700009DC7000044
:100020009BC7000099C7000097C7000095C7000054
:1000300093C7000091C700008FC700008DC7000064
:100040008BC7000089C7000087C7000085C7000074
:1000500083C7000081C700007FC700000C94680BB5
:100060007BC700000C94350A0C940C0A75C700007D
:1000700073C7000071C700006FC700006DC70000A4
:100080006BC7000069C7000067C7000065C70000B4
:1000900063C7000061C700005FC700000C94B20B8B
:1000A0005BC7000059C7000057C7000055C70000D4
:1000B00053C7000051C700004FC700004DC70000E4
:1000C0004BC7000049C7000047C7000045C70000F4
:1000D00043C7000041C700003FC700003DC7000004
:1000E0003BC700009A0A9D0A8C0A900A940AD40A17
:1000F000A10AA50AAB0AAF0AB30AB90ABD0AC10A26
:10010000D40AC70ACB0ACF0A762B7C2B832B8A2BE7
:100110009D2BB02BC32B00002100240027002A00B8
:100120002D003000330001010000040107010A0125
:1001300001021020200808102040102040800201F9
:1001400002010804020101020408102040808040DE
:1001500020100804020180040201804020100804DD
:10016000020108040201010204081020408001027B
:100170000408102040800505050507050808080843
:10018000020202020A0A080804040404010101012F
:10019000010101010303030303030303040707072A
:1001A0000C0C0C0C0C0C0C0C0202020206060606CF
:1001B000060606060B0B0B0B0B0B0B0B47422046E0
:1001C000415400534420436172643A200053442058
:1001D0004572726F720A00496E697469616C697A5E
:1001E000696E6720534420636172642E2E2E005680
:1001F000422050726F6772616D6D6572206C697616
:100200006573210A0047616D652056657273696FD9
:100210006E3A20312E0047616D6520436F64653A68
:1002200020004D616B657220436F64653A20004782
:10023000616D65205469746C653A20002A2A2A2A67
:100240002A2A2A2A2A2A2A2A2A2A2A2A2A2A2A2A0E
:100250002A2A2A2A2A2A2A2A2A2A2A2A2A2A2A2AFE
:100260002A2A2A2A2A2A2A2A2A2A2A2A2A2A2A2AEE
:100270002A2A2A2A2A2A2A2A2A2A2A2A2A2A2A2ADE
:100280002A2A2A00575252202020202020202020D5
:10029000202020202020202057726974652053528E
:1002A000414D005752462020202020202020202091
:1002B00020202020202020577269746520466C6120
:1002C0007368005652462020202020202020202025
:1002D0002020202020202056657269667920466CF7
:1002E00061736820636F6E74656E74730056455257
:1002F00020202020202020202020202020202020FE
:10030000205072696E742076657273696F6E206F0B
:10031000662070726F6772616D6D657220666972BA
:100320006D776172650053444620202020202020F4
:100330002020202020202020202053656C6563741D
:1003400020534420636172642066696C652070618B
:10035000746820666F722070726F6772616D6D696C
:100360006E67005352532020202020202020202080
:1003700020202020202020536574205352414D20FE
:100380006269742073697A6520746F20706F776575
:1003900072206F6620325E2831362C31382C323292
:1003A000206F6E6C79290053465320202020202096
:1003B000202020202020202020202053657420464B
:1003C0006C617368206269742073697A6520746F48
:1003D00020706F776572206F6620325E2832342C71
:1003E00032372C3238206F6E6C792900534320202D
:1003F00020202020202020202020202020202020FD
:100400005365747570204361727420706F727473D9
:1004100020666F7220726561642F7772697465005F
:100420005253542020202020202020202020202033
:1004300020202020526573657420466C617368002B
:1004400048525354202020202020202020202020EB
:1004500020202020536F66747761726520465720F4
:10046000526573746172740052445220202020201F
:100470002020202020202020202020205265616480
:10048000205352414D00524446202020202020205D
:10049000202020202020202020205265616420463A
:1004A0006C61736800524441542020202020202099
:1004B00020202020202020202052656164206461BB
:1004C00074612070696E732028646562756767695E
:1004D0006E67290052414444202020202020202003
:1004E0002020202020202020526561642061646447
:1004F000726573732070696E732028646562756716
:1005000067696E6729005052425220202020202027
:10051000202020202020202020205072696E74206E
:100520005352414D20636F6E74656E747320696E13
:100530002062696E6172790050524246202020206C
:100540002020202020202020202020205072696E92
:100550007420666C61736820636F6E74656E74736B
:1005600020696E2062696E61727900505254462093
:10057000202020202020202020202020202020504B
:1005800072696E7420666C61736820636F6E746547
:100590006E747320696E20415343494900504D20C9
:1005A000202020202020202020202020202020204B
:1005B000205072696E742074686973206D656E7561
:1005C00000494446202020202020202020202020D8
:1005D00020202020205072696E74204944206F66CC
:1005E00020466C6173680045535F5820202020200E
:1005F000202020202020202020202053657420450A
:1006000053206C696E652031206F72203000455296
:1006100052202020202020202020202020202020A8
:1006200020204572617365205352414D004552466A
:1006300020202020202020202020202020202020BA
:1006400020457261736520466C61736800444154B3
:10065000415F58585858202020202020202020205A
:100660002053657420646174612070696E73207416
:100670006F20306858585F58580042434620202069
:100680002020202020202020202020202020426CFC
:10069000616E6B20436865636B20466C6173680014
:1006A0004155544F20202020202020202020202091
:1006B000202020204175746F2050726F6772616D29
:1006C0002E2045726173652C20426C616E6B204355
:1006D0006865636B2C2057726974652C20566572AF
:1006E00069667900414444525F5858585858582018
:1006F0002020202020202020536574206164647213
:100700006573732070696E7320746F203068585859
:100710005F58585F5858002D2D2D2D2D2D2D2D2D26
:100720002D2D2D2D2D2D2D2D2D2D2D2D2D2D2D2DF9
:100730002D2D2D2D2D2D2D2D2D2D2D2D2D2D2D2DE9
:100740002D2D2D2D2D2D2D2D2D2D2D2D2D2D2D2DD9
:100750002D2D2D2D2D2D2D2D2D2D2D2D2D2D2D00F6
:10076000436F6D6D616E64202020202020202020AA
:10077000202020204465736372697074696F6E0075
:100780002A2A2A2A2A2A2A2A2A2A2A2A2A2A2A2AC9
:100790002A2A2A2A2A2A2A2A2A2A56422050726FCC
:1007A0006772616D6D6572204D656E752A2A2A2A01
:1007B0002A2A2A2A2A2A2A2A2A2A2A2A2A2A2A2A99
:1007C0002A2A2A2A2A2A2A2A005352414D205772BD
:1007D00069746520436F6D706C65746564210043B6
:1007E000616E2774206F70656E2066696C65206F7E
:1007F0006E2053442E0046696C652073697A65202B
:100800006578636565647320666C617368207369DD
:100810007A652E0057726974696E672066696C6527
:100820003A200057726974696E67205352414D2E09
:100830002E2E0046696E6973686564207265616476
:10084000696E6720466C6173682E0043616E277481
:10085000206372656174652066696C65206F6E2027
:1008600053442E00536176696E6720746F205344A1
:100870002061733A200052656164696E6720466C9E
:100880006173682E2E2E0046696E69736865642058
:1008900072656164696E67205352414D2E00436159
:1008A0006E2774206372656174652066696C6520CB
:1008B0006F6E2053442E00536176696E6720746F0B
:1008C0002053442061733A200052656164696E6769
:1008D000205352414D2E2E2E0045726173652043E8
:1008E0006F6D706C65746564210045726173696E2B
:1008F0006720466C617368004F7065726174696F40
:100900006E20746F6F6B203A20004E6F7420612050
:1009100076616C69642073697A6520666F7220461F
:100920006C6173682E2044656661756C74696E67CE
:1009300020746F2031364D6269742028322C303992
:10094000372C313532206279746573292E00536556
:100950007474696E6720466C6173682053697A65A8
:100960003A20004E6F7420612076616C69642073B8
:10097000697A6520666F72205352414D2E2044657E
:100980006661756C74696E6720746F20386B2078AF
:100990002038202836352C353336204D62697429AD
:1009A0002E0053657474696E67205352414D205375
:1009B000697A653A200052656164696E6720476113
:1009C0006D65204865616465720052656164696E99
:1009D0006720416464726573732070696E733A2096
:1009E0000053657474696E67204461746120706996
:1009F0006E7320746F3A200053657474696E6720BB
:100A0000416464726573732070696E7320746F3A09
:100A10002000536574757020444F4E450053657433
:100A200074696E6720757020666C61736820696EEA
:100A300074657266616365005265736574696E679B
:100A400020666C6173682E2E2E005072696E746978
:100A50006E67205352414D20696E204153434949EE
:100A6000005072696E74696E6720666C61736820ED
:100A7000696E2041534349490052656164696E675C
:100A8000205352414D2E2E2E00446174613A2000B5
:100A9000454550524F4D20436C65617220436F6D48
:100AA000706C6574656400436C656172696E672083
:100AB000454550524F4D0000002200250028002BD4
:100AC000002E003100340002010000050108010B76
:100AD0000100000A0B02090C0D0E080703040100B7
:100AE0000000000000000000000000000000000006
:100AF00000000000000000000000000000121110C3
:100B000000000000000000000000000000000000E5
:100B100000000000000000556E6B6E6F776E20665F
:100B20006C617368726F6D004379707265737320C6
:100B3000533239474C323536502F53206465746533
:100B4000637465640043797072657373205332393E
:100B5000474C313238502F53206465746563746597
:100B600064004D6963726F6E204D323957323536ED
:100B70004748206465746563746564004D696372F9
:100B80006F6E204D323957313238474820646574D2
:100B90006563746564004D6163726F6E6978204DA2
:100BA0005832394631363130206465746563746576
:100BB00064004465766963652049442057333A20D0
:100BC000004465766963652049442057323A200025
:100BD0004465766963652049442057313A20004DC9
:100BE000616E662E2049443A20004572617365208B
:100BF000436F6D706C657465642100506C65617342
:100C00006520776169742E2E2E0045726173696EBE
:100C100067004572726F723A204E6F7420626C6189
:100C20006E6B00426C616E6B20436865636B205095
:100C300061737365642100506C6561736520776131
:100C400069742E2E2E00426C616E6B2043686563C2
:100C50006B0050726F6772616D6D696E6720436FD4
:100C60006D706C65746564210050726F6772616DA0
:100C70006D696E67204552524F52210043616E27C5
:100C800074206F70656E2066696C65206F6E2053EE
:100C9000442E0046696C652073697A6520646F652F
:100CA00073204E4F5420657175616C20666C6173C2
:100CB000682073697A652E0057726974696E6720BF
:100CC0004D583239463136313020466C6173682ECA
:100CD0002E2E00466C617368696E672066696C65CC
:100CE0003A200050726F6772616D6D696E672043C4
:100CF0006F6D706C65746564210043616E277420AC
:100D00006F70656E2066696C65206F6E2053442E8F
:100D10000046696C652073697A6520646F6573208D
:100D20004E4F5420657175616C20666C617368204C
:100D300073697A652E0057726974696E6720466C14
:100D40006173682E2E2E00466C617368696E672091
:100D500066696C653A200050726F6772616D6D69EB
:100D60006E6720436F6D706C65746564210043612C
:100D70006E2774206F70656E2066696C65206F6EDB
:100D80002053442E0046696C652073697A6520649F
:100D90006F6573204E4F5420657175616C20666CD1
:100DA0006173682073697A652E0057726974696E81
:100DB0006720466C6173682E2E2E00466C61736846
:100DC000696E672066696C653A20005665726966CF
:100DD00069636174696F6E2050415353454421002B
:100DE0005344204275666665723A2000466C617312
:100DF000683A200043757272656E7420506F733AC2
:100E00002000566572696669636174696F6E20457A
:100E100052524F52210043616E2774206F70656EED
:100E20002066696C65206F6E2053442E0046696C05
:100E3000652073697A6520657863656564732066EB
:100E40006C6173682073697A652E005665726966F5
:100E500079696E6720466C6173682E2E2E00466C91
:100E6000617368726F6D20577269746572203136D4
:100E700062697400616E6420656E74657220612021
:100E800073656C656374696F6E2062792074797024
:100E9000696E672061206E756D62657228302D362F
:100EA000293A205F2000506C656173652062726F83
:100EB0007773652070616765732077697468202790
:100EC00075272875702920616E642027642728649F
:100ED0006F776E2900290046696C6562726F7773BF
:100EE00065723A2000546F6F206D616E79206669DB
:100EF0006C6573000C3F11241FBECFEFD1E2DEBF43
:100F0000CDBF00E00CBF14E0A0E0B2E0E8E8FAE8F2
:100F100000E00BBF02C007900D92AC35B107D9F7C6
:100F20002DE0ACE5B4E001C01D92A23CB207E1F7B0
:100F300017E0CBE7D7E000E006C021970109802F3A
:100F4000FE010E942642CA37D10780E00807A9F7B0
:100F50000E94A62F0C94424553C8CF92DF92EF9285
:100F6000FF920F931F93CF93DF936C017A018B0154
:100F7000C0E0D0E0CE15DF0589F0D8016D918D017C
:100F8000D601ED91FC910190F081E02DC6011995FB
:100F9000892B11F47E0102C02196ECCFC701DF91AD
:100FA000CF911F910F91FF90EF90DF90CF90089518
:100FB000FC01538D448D252F30E0842F90E0821B5F
:100FC000930B541710F0CF96089501970895FC01E4
:100FD000918D828D981761F0828DDF01A80FB11D70
:100FE0005D968C91928D9F5F9F73928F90E0089594
:100FF0008FEF9FEF0895FC01918D828D981731F04E
:10100000828DE80FF11D858D90E008958FEF9FEFA1
:101010000895FC01918D228D892F90E0805C9F4F77
:10102000821B91098F739927089589E99AE0F1DF6E
:1010300021E0892B09F420E0822F0895FC01848DA2
:10104000DF01A80FB11DA35ABF4F2C91848D90E0F2
:1010500001968F739927848FA689B7892C93A089CD
:10106000B1898C9180648C93938D848D981306C084
:101070000288F389E02D80818F7D80830895EF922F
:10108000FF920F931F93CF93DF93EC0181E0888F42
:101090009B8D8C8D981305C0E889F989808185FD29
:1010A00023C0F62E0B8D10E00F5F1F4F0F7311271B
:1010B000E02E8C8DE8120BC00FB607FCFACFE88942
:1010C000F989808185FFF5CFCE01B8DFF2CF8B8D16
:1010D000FE01E80FF11DE35AFF4FF0820B8FEA8902
:1010E000FB898081806207C0EE89FF896083E8897F
:1010F000F98980818064808381E090E0DF91CF91E5
:101100001F910F91FF90EF900895CF93DF93EC0123
:10111000888D8823C1F0EA89FB89808185FD05C01F
:10112000A889B9898C9186FD0EC00FB607FCF5CF52
:10113000808185FFF2CFA889B9898C9185FFEDCF99
:10114000CE017CDFE8CFDF91CF91089580E090E081
:10115000892B19F06ADF811125C080E090E0892B8E
:1011600041F080E090E0892B21F00E940000811185
:101170001CC080E090E0892B41F080E090E0892B5A
:1011800021F00E940000811113C080E090E0892BC3
:10119000A1F080E090E0892B81F00E940000811195
:1011A0000AC008950E940000D8CF0E940000E1CF3D
:1011B0000E940000EACF0C94000008953FB7F89415
:1011C0008091A0079091A107A091A207B091A307D9
:1011D00026B5A89B05C02F3F19F00196A11DB11D92
:1011E0003FBFBA2FA92F982F8827820F911DA11DCD
:1011F000B11DBC01CD0142E0660F771F881F991F0A
:101200004A95D1F7089585ED8093BC008091BC008C
:1012100084FDFCCF10923308089540915207262F89
:1012200030E0240F311D21323105DCF420913308E8
:101230002430C9F4FC0180E090E0861758F4309126
:1012400052072191DC01A05DB84FA30FB11D2C9373
:101250000196F3CF80915207680F6093520780E0A8
:10126000089581E0089582E00895089581E090E076
:101270003091370820913608321710F480E090E062
:10128000919581959109089580913708909136083C
:10129000891730F48F5F8093370880E090E00895DD
:1012A0008FEF9FEF08958091360890E020913708E6
:1012B000821B91090895CF92DF92EF92FF920F93D4
:1012C0001F93CF93DF937C01262F972F8A01809164
:1012D0002F07882391F0C62FD72F6E01C40ED51E7D
:1012E000CC15DD0569F06991D701ED91FC91019074
:1012F000F081E02DC7011995F3CF642F822F8DDF88
:10130000C801DF91CF911F910F91FF90EF90DF9077
:10131000CF900895CF93DF931F92CDB7DEB7698347
:1013200020912F072223D1F020913408203240F061
:1013300021E030E0FC013383228380E090E014C0A0
:1013400080913508E82FF0E0E15FF84F99819083B4
:101350008F5F809335088093340804C061E0CE012C
:1013600001965BDF81E090E00F90DF91CF910895CF
:101370000E942E424F925F926F927F92EF92FF9265
:101380000F931F93CF93DF93CDB7DEB7A1970FB61F
:10139000F894DEBF0FBECDBF7C01FA01CB0119A2CC
:1013A000223008F42AE08E010F5D1F4F422E512C8F
:1013B000612C712CBF01A30192010E94C73FF9016A
:1013C000CA01015011096A3014F4605D01C0695C02
:1013D000D8016C93232B242B252B61F7B801C7016F
:1013E0000E942F1DA1960FB6F894DEBF0FBECDBF91
:1013F000DF91CF911F910F91FF90EF907F906F90B1
:101400005F904F900895DC01ED91FC910190F08187
:10141000E02D19940C942F1D1F920F920FB60F926E
:1014200011240BB60F922F933F934F935F936F93BB
:101430007F938F939F93AF93BF93EF93FF9389E92C
:101440009AE0FCDDFF91EF91BF91AF919F918F9159
:101450007F916F915F914F913F912F910F900BBEB4
:101460000F900FBE0F901F9018951F920F920FB6FE
:101470000F9211240BB60F922F938F939F93EF939C
:10148000FF93E091A90AF091AA0A8081E091AF0A46
:10149000F091B00A82FD12C090818091B20A8F5FF4
:1014A0008F732091B30A821751F0E091B20AF0E0F5
:1014B000E756F54F958F8093B20A01C08081FF9166
:1014C000EF919F918F912F910F900BBE0F900FBEB8
:1014D0000F901F901895362F90E0FC01EF52F54FBA
:1014E0004491FC01E05DFE4F2491FC01EA58FE4F5F
:1014F0009491992309F46BC0442309F455C050E03A
:10150000FA013197E231F10508F04EC08827EE5814
:10151000FF4F8F4F0C942642809180008F7707C039
:10152000809180008F7D03C080918000877F8093B1
:1015300080003AC084B58F7702C084B58F7D84BDAA
:1015400033C08091B0008F7703C08091B0008F7D51
:101550008093B00029C0809190008F7707C0809160
:1015600090008F7D03C080919000877F80939000D2
:101570001BC08091A0008F7707C08091A0008F7D55
:1015800003C08091A000877F8093A0000DC0809150
:1015900020018F7707C0809120018F7D03C080914B
:1015A0002001877F80932001E92FF0E0EE0FFF1FDD
:1015B000E954F54FA591B4918FB7F894EC9131119E
:1015C00003C020952E2301C02E2B2C938FBF08958E
:1015D000CF93DF9390E0FC01E05DFE4F2491FC018E
:1015E000EA58FE4F8491882361F190E0880F991F9B
:1015F000FC01EA5EFE4FC591D491FC01E954F54F20
:10160000A591B491611109C09FB7F8948881209584
:1016100082238883EC912E230BC0623061F49FB744
:10162000F8943881822F809583238883EC912E2B28
:101630002C939FBF06C08FB7F894E8812E2B288388
:101640008FBFDF91CF9108958F929F92AF92BF92FB
:10165000CF92DF92EF92FF926B017C01AFDD4B01E5
:101660005C01C114D104E104F104E9F0A7DDDC015F
:10167000CB0188199909AA09BB09883E9340A105A5
:10168000B10578F321E0C21AD108E108F10888EE2B
:10169000880E83E0981EA11CB11CC114D104E10482
:1016A000F10421F7DECFFF90EF90DF90CF90BF9055
:1016B000AF909F908F9008952FB7F89460919C07FA
:1016C00070919D0780919E0790919F072FBF08956D
:1016D0001F920F920FB60F9211242F933F938F9367
:1016E0009F93AF93BF9380919C0790919D07A0918A
:1016F0009E07B0919F0730919B0723E0230F2D3762
:1017000020F40196A11DB11D05C026E8230F029605
:10171000A11DB11D20939B0780939C0790939D076B
:10172000A0939E07B0939F078091A0079091A10777
:10173000A091A207B091A3070196A11DB11D8093AE
:10174000A0079093A107A093A207B093A307BF910E
:10175000AF919F918F913F912F910F900FBE0F905E
:101760001F9018951F920F920FB60F9211240BB66F
:101770000F922F933F934F935F936F937F938F932A
:101780009F93AF93BF93EF93FF938091B900887FAE
:10179000803609F49CC068F5883209F45BC090F487
:1017A000803109F454C038F4882309F4F6C0883035
:1017B00009F44DC0F5C0883109F44CC0803209F4F9
:1017C0005DC0EEC0803409F468C048F4803309F489
:1017D00055C0883309F0E4C080937707D8C08035BE
:1017E00009F44FC0883509F45DC0883409F0D8C0C9
:1017F000D6C0883909F4C7C0A8F4883709F467C08F
:1018000038F4883609F463C0803709F460C0C8C072
:10181000883809F4B8C0803909F45FC0803809F00D
:10182000BFC05BC0803B09F486C038F4803A09F43D
:1018300066C0883A09F47FC0B3C0803C09F4A7C0F1
:10184000883C09F4A4C0883B09F48AC0A9C08091EF
:101850009A0710C09091990780919807981770F592
:10186000E091990781E08E0F80939907F0E0E858A6
:10187000F84F80818093BB0085EC86C0809377070A
:101880008EC0E091990781E08E0F80939907809137
:10189000BB00F0E0E858F84F808390919907809161
:1018A00098076EC0E091990781E08E0F80939907A9
:1018B0008091BB00F0E0E858F84F808380913208B7
:1018C00081116DC081E08093310884EA61C083E0BA
:1018D0008093330810927607CFCF809176078032BD
:1018E00008F051C0E091760781E08E0F8093760773
:1018F0008091BB00F0E0EA5AF84F8083BDCF85ECC1
:101900008093BC001092330880917607803230F4C7
:10191000E0917607F0E0EA5AF84F1082609176077E
:1019200070E0E0915407F091550786E597E019952E
:101930001092760735C084E08093330810925307E5
:1019400010925207E0915007F0915107199580913C
:101950005207811105C081E0809352071092300731
:10196000E091530781E08E0F80935307F0E0E05D34
:10197000F84F80818093BB0090915307809152076C
:10198000981708F479CF85E88093BC0009C085ECEE
:101990008093BC001092330803C01092770733DCA9
:1019A000FF91EF91BF91AF919F918F917F916F9137
:1019B0005F914F913F912F910F900BBE0F900FBEF3
:1019C0000F901F901895CF93FC01C48121E02093C4
:1019D0002F07C0930E0710923508109234088385A4
:1019E000682B86E39BE096DC80913408813208F016
:1019F00046C0909133089111FCCF92E09093330848
:101A000091E0909332089FEF909377071092990797
:101A100080939807AFE0B7E028E737E0F9019E2F01
:101A2000921B981718F49D919193F9CF10929A07F1
:101A300080919A07CC0FC82BC0939A0780913108E8
:101A4000813061F41092310880919A078093BB0035
:101A50008091BC0083FDF8CF85EC01C085EE8093BA
:101A6000BC00809133088230E1F3809177078F3F8B
:101A700031F080917707803211F0809177071092D2
:101A800035081092340810922F07CF9108950F93C4
:101A90001F93CF938C01C62F96DF6C2F6460C80113
:101AA00092DF6C2F6B7FC8018EDF83EC90E0019793
:101AB000F1F7CF911F910F9108950F931F93CF933B
:101AC0008C01C62F607F6160E2DF80E1C89FB001BA
:101AD00011246160C801DBDF81E090E0CF911F91AC
:101AE0000F9108958EBD0DB407FEFDCF08958FEFC1
:101AF0008EBD0DB407FEFDCF8EB50895CF93DF9355
:101B0000FC012381222351F0EC010180F281E02DC0
:101B100061E08281E0DC8FEFE5DF1B82DF91CF9116
:101B200008950F931F93CF93DF938C01862FEA01C3
:101B3000D9DF88818EBD8981FE013296DE5F0DB4CA
:101B400007FEFDCF8EBDEC17FD0711F08191F7CF99
:101B50000DB407FEFDCF8FEFC5DF8FEFC3DFC7DF0B
:101B6000F8018483982F9F71953031F087E5808349
:101B7000C801C4DF80E001C081E0DF91CF911F91F7
:101B80000F9108950F931F93CF93DF93EC01890179
:101B90008D81833039F089E0440F551F661F771F10
:101BA0008A95D1F79A01AB0168E1CE010E944A1BE8
:101BB000882311F082E31DC0A8016EEFCE01B1DFD2
:101BC0008823C1F00E94062C182F811102C08AE5DB
:101BD00010C020E030E0A9016DE0CE010E944A1B58
:101BE000811106C084DF811103C0CE0187DF05C0EB
:101BF00089E28883CE0182DF10E0812FDF91CF91CF
:101C00001F910F910895089580E090E00895049643
:101C10000C940317CF93DF931F92CDB7DEB7698380
:101C200041E050E0BE016F5F7F4F04960E940317B2
:101C30000F90DF91CF91089504960C94C91680E01F
:101C40000C948D2E81E00C948D2E31E020E07F9B52
:101C500030E0832F922F2091090124FD826030997A
:101C600084600799886001998061369980629299B1
:101C700080642091090122FD80682091090120FDE6
:101C80009160909992603499946003999860059955
:101C90009061329990622091090126FD90647D99AE
:101CA000906808952091080160FF02C0226001C081
:101CB0002D7F2093080161FF02C0A59A01C0A5985D
:101CC00062FF02C05A9A01C05A982091020163FF34
:101CD00002C0216001C02E7F2093020164FF02C078
:101CE000749A01C0749865FF02C08E9A01C08E98E4
:101CF00020910B0166FF02C0226001C02D7F20935E
:101D00000B0120910B0167FF02C0206201C02F7DF3
:101D100020930B0170FF02C08C9A01C08C9871FF58
:101D200002C0759A01C075982091020172FF02C02D
:101D3000226001C02D7F2093020173FF02C05B9AD5
:101D400001C05B9874FF02C0739A01C07398209120
:101D5000080175FF02C0216001C02E7F2093080199
:101D60002091080176FF02C0246001C02B7F2093E0
:101D700008012091080177FF02C0206101C02F7E79
:101D8000209308012091080180FF02C0206201C059
:101D90002F7D2093080181FF02C0A19A01C0A19864
:101DA00082FF02C0419A01C0419820910B0183FF3C
:101DB00002C0286001C0277F20930B0120910B01F6
:101DC00084FF02C0206801C02F7720930B0185FF9C
:101DD00002C05F9A01C05F9886FF02C0439A0895CF
:101DE00043980895CF93DF93169800005BDF0000BF
:101DF000C8E0D1E088818F7B88830000000000006C
:101E000000000000000021DF9C0100009881906428
:101E10009883000000000000000000000000169AF7
:101E20000000C901DF91CF910895CF93DF93EA01BC
:101E30001698000037DFCE010E94D02E00001098C7
:101E4000000000000000000000000000109A0000E8
:101E500000000000000000000000169A0000DF9162
:101E6000CF910895CF93DF93C8E0D1E02881277FF9
:101E70002883000017DF000088818F7B88830000A3
:101E800000000000000000000000DFDE9C010000F8
:101E9000988190649883000000000000000000001A
:101EA00000009881986098830000C901DF91CF916C
:101EB0000895CF93DF931F921F92CDB7DEB7BFDE99
:101EC00060E070E0CB01CEDF87FFFACF89839A8391
:101ED000B9DE89819A810F900F90DF91CF9108959B
:101EE0000F931F93CF93DF938A01C8E0D1E028813D
:101EF000277F28830000D6DEC8010E94D02E000074
:101F00001498000000000000000000000000149A77
:101F100000000000000000000000000088818860D0
:101F200088830000DF91CF911F910F910895CF9387
:101F3000DF9388DE8091600682504AEA50E0843068
:101F400098F065E575E580E090E0CADF45E550E092
:101F50006AEA7AE280E090E0C3DF40E950E065E5BC
:101F600075E580E090E012C065E575E080E090E006
:101F7000B7DF45E550E06AEA72E080E090E0B0DF6C
:101F800040E950E065E575E080E090E0A9DF57DECC
:101F900060E070E0CB0166DF9F938F93C6EBD3E0E8
:101FA000DF93CF9382ED97E09F938F930E947642C9
:101FB00061E070E080E090E055DF9F938F93DF93C6
:101FC000CF9383EC97E09F938F930E9476426EE0CD
:101FD00070E080E090E046DF9F938F93DF93CF9394
:101FE00084EB97E09F938F930E9476426FE070E0BE
:101FF00080E090E037DF9F938F93DF93CF9385EA64
:1020000097E09F938F930E9476428FED9BE00E9412
:10201000312F82ED97E00E94612F80ED9BE00E94BE
:10202000312F83EC97E00E94612F81EC9BE00E94AE
:10203000312F84EB97E00E94612F82EB9BE00E949E
:10204000312F85EA97E00E94612F6BEB73E082ED00
:1020500097E00E9466422DB73EB7285E3F4F0FB60D
:10206000F8943EBF0FBE2DBF892B59F460EC73E08E
:1020700083EC97E00E946642892B19F486E99BE085
:102080005FC065EC73E082ED97E00E946642892BA9
:1020900029F56AEC73E084EB97E00E946642892B95
:1020A00019F48CE79BE00AC06FEC73E084EB97E0D7
:1020B0000E946642892B91F482E69BE00E94522F97
:1020C00080E090E0A0E0B1E080934A0290934B0260
:1020D000A0934C02B0934D0282E02CC064ED73E0FB
:1020E00082ED97E00E946642892B41F56AEC73E02D
:1020F00084EB97E00E946642892B19F485E49BE00B
:102100000AC06FEC73E084EB97E00E946642892B73
:10211000A9F488E29BE00E94522F80E090E0A0E0CA
:10212000B1E080934A0290934B02A0934C02B0938B
:102130004D0284E08093600681E013C087E19BE05C
:102140000E94522F80E090E0A0E2B0E080934A022B
:1021500090934B02A0934C02B0934D0281E0809388
:1021600060068093A40780E090E2909349028093F8
:10217000480288EE93E0DF91CF910C94612F62DDED
:10218000809160068130A9F44AEA50E065E575E582
:1021900080E090E0A5DE45E550E06AEA7AE280E082
:1021A00090E09EDE40EF50E065E575E580E090E070
:1021B00017C082508430A8F44AEA50E065E575E023
:1021C00080E090E08DDE45E550E06AEA72E080E074
:1021D00090E086DE40EF50E065E575E080E090E05D
:1021E0007FDE2DDD64EF71E080E090E02DCA20916C
:1021F0000801277F20930801000054DD0000809132
:1022000008018F7B8093080100000000000000009F
:102210000000000031E020E07F9B30E0832F922F10
:102220002091090124FD82603099846007998860BB
:1022300001998061369980629299806420910901A8
:1022400022FD80689091080190649093080100003D
:1022500090910801986090930801000008956EE93C
:1022600072E080E00E942E2E66E972E081E00E941A
:102270002E2E6EE872E082E00E942E2E60E172E067
:1022800083E00E942E2E68E072E084E00E942E2EF1
:1022900060E072E085E00E942E2E66E872E086E043
:1022A0000C942E2E0F931F93CF93DF938C01EB0191
:1022B0000E94862ED4DF82E00E941D2EEBE3FFE118
:1022C0003197F1F760E080E00E945B2EB80186EB69
:1022D0009DE0A0D861E080E00E945B2EBE0186EB0D
:1022E0009DE098D860E08DE00E945B2E60E086EB78
:1022F0009DE0E3DB61E086EB9DE0DFDB62E086EB07
:102300009DE0DBDB61E08DE00E945B2E63E086EB0D
:102310009DE0D3DB64E086EB9DE0CFDB65E086EB00
:102320009DE0DF91CF911F910F91C7CB1F93CF936A
:10233000DF938AE09CE00E94522F8BEF9BE00E948B
:10234000312F60E080E00E945B2E69ED73E086EB48
:102350009DE060D861E080E00E945B2E6AEE73E051
:1023600086EB9DE057D86EDC80916006813051F598
:102370004AEA50E065E575E580E090E0B1DD45E5CD
:1023800050E06AEA7AE280E090E0AADD40E850E0BE
:1023900065E575E580E090E0A3DD4AEA50E065E59B
:1023A00075E580E090E09CDD45E550E06AEA7AE280
:1023B00080E090E095DD40E150E065E575E580E086
:1023C00090E02CC08250843050F54AEA50E065E538
:1023D00075E080E090E084DD45E550E06AEA72E077
:1023E00080E090E07DDD40E850E065E575E080E06C
:1023F00090E076DD4AEA50E065E575E080E090E047
:102400006FDD45E550E06AEA72E080E090E068DD6B
:1024100040E150E065E575E080E090E061DD0FDCD3
:1024200080916006813011F444DD1FC082508430F9
:10243000E0F405DC60E070E0CB0114DD182FC0E0B3
:10244000D0E017FD11C060E070E0CB010BDD182F6C
:10245000CE019370892B31F46AE973E089E99AE03F
:102460000E940A0A2196EDCFEDDB88E093E00E94FE
:10247000612F8AEE9BE00E94522F63E173E08EE1B0
:1024800093E0DF91CF911F910DCFCF93DF93C82FB2
:1024900060E08CE00E945B2E4C2F50E060E070E02A
:1024A00086EB9DE00E94742F6BEF73E086EB9DE05E
:1024B0000E940A0A61E080E00E945B2E2C2F30E02F
:1024C000AEE1B0E00E94E93F24E630E040E050E0B9
:1024D0000E94A13FC22FD0E0D1110AC0CC2331F01D
:1024E00061E086EB9DE0E9DAC1501EC060E005C006
:1024F000DF3049F4CC2329F066E086EB9DE0DDDA9D
:1025000013C065E0FACFC23030F064E086EB9DE0A6
:10251000D4DAC25009C0C13011F463E001C062E0F6
:1025200086EB9DE0CADAC0E0DF5FD031A9F6DF912B
:10253000CF910895CF93DF93EC016EE772E080E0D6
:102540000E942E2E66E772E081E00E942E2E6EE63B
:1025500072E082E00E942E2E66E672E083E00E9426
:102560002E2E6EE572E084E00E942E2E66E572E06B
:1025700085E00E942E2E6EE472E086E00E942E2EF0
:102580000E94862E60E080E00E945B2EBE0186EBFA
:102590009DE0DF91CF910C940A0A4F925F926F9267
:1025A0007F928F929F92AF92BF92CF92DF92EF92E3
:1025B000FF920F931F93CF93DF93EC014A015B01CE
:1025C0004C845D846E847F84A881AA2309F491C021
:1025D000488959896A897B8984169506A606B706B3
:1025E00009F48DC081149104A104B10429F41C865E
:1025F0001D861E861F8678C0A3FF0BC0088D198D0F
:102600002A8D3B8D081519052A053B0508F471C074
:1026100014C0A5FF12C0EE81FF818681978125E05D
:10262000880F991F2A95E1F7A0E0B0E08815990579
:10263000AA05BB0508F45DC057C0EE81FF81848107
:1026400090E009968A019B01015011092109310985
:10265000082E04C036952795179507950A94D2F74A
:1026600075016401B1E0CB1AD108E108F10804C09A
:10267000F694E794D794C7948A95D2F7C016D106FA
:10268000E206F30620F0452B462B472B81F4A6FFEC
:1026900005C0848D958DA68DB78D04C08C8D9D8DC4
:1026A000AE8DBF8D8C879D87AE87BF8704C0C01A53
:1026B000D10AE20AF30A8E01045F1F4FC114D1044C
:1026C000E104F10489F04C855D856E857F85980174
:1026D0008E819F810E94B21C91E0C91AD108E10845
:1026E000F10818165CF305C0888A998AAA8ABB8A01
:1026F00006C04C865D866E867F8680E001C081E0E4
:10270000DF91CF911F910F91FF90EF90DF90CF90CD
:10271000BF90AF909F908F907F906F905F904F9001
:1027200008953F924F925F926F927F928F929F9205
:10273000AF92BF92CF92DF92EF92FF920F931F93CF
:10274000CF93DF93CDB7DEB728970FB6F894DEBFEF
:102750000FBECDBF98878F835B018A01DC018C910E
:10276000882309F112969C9190FF1DC027C03380E9
:102770003422C114D10409F098C0311096C0892BBD
:102780008A2B8B2B09F47AC0AF81B8851C964D91AA
:102790005D916D917C911F9729813A81C4010E94BE
:1027A000B21C87FF7AC0AF81B88511968C911197C2
:1027B000826011968C938FEF9FEF67C183FF17C0E4
:1027C000EF81F885808D918DA28DB38D40895189DF
:1027D00062897389841B950BA60BB70BA80160E077
:1027E00070E0481759076A077B07D0F018C085FFCB
:1027F00017C0AF81B8851696ED91FC911797868129
:102800009781F5E0880F991FFA95E1F750962D9181
:102810003C915197821B930B8017910708F48C0110
:102820007801312CEF81F8853C96FA83E983E11435
:10283000F10409F477C0EF81F88580899189A28934
:10284000B3896C01F1E0DF22EF81F8852081868079
:102850009780AC01BD01E9E076956795579547955E
:10286000EA95D1F7F40125FF82CF848D958DA68D51
:10287000B78D480F591F6A1F7B1F3BC026FD02C042
:10288000EF81F885848D958DA68DB78DEF81F885C4
:1028900084879587A687B78708C0811106C0EF8116
:1028A000F88580818077F1F57ECFAF81B885169667
:1028B000ED91FC9117971C964D915D916D917C91D6
:1028C0001F974250510961097109048004C0440FE7
:1028D000551F661F771F0A94D2F780899189A289B4
:1028E000B389480F591F6A1F7B1F430D511D611D7E
:1028F000711DAF81B8851696ED91FC911797C114A3
:10290000D10409F09CC0E114B2E0FB0608F497C0C2
:1029100063A074A085A096A04615570568057905A3
:1029200029F48DC0C8018E199F09AFC0E114B4E02D
:10293000FB0608F467C02701452C55244694AF8157
:10294000B8858C9185FD07C08281831990E084153C
:10295000950508F42C016416750686069706A0F402
:10296000AF81B8851696ED91FC911797C080D18004
:10297000F60185818330A9F029E0440F551F661FB9
:10298000771F2A95D1F70DC0D401C301840D951D81
:10299000A11DB11D481759076A077B0708F467C0D6
:1029A000DFCF9A01AB0162E1C60174D6811104C088
:1029B0003501812C912C0FC081E319C040E052E019
:1029C000B301C60115D6882309F4EDCEBFEF8B1AEB
:1029D0009B0AEEEF7E1A8414950481F720E030E024
:1029E000A9016CE0C60156D6882331F088E2D601F1
:1029F0008C93C60183D8D7CE982C8824990CC60115
:102A00007DD80AC09501808191818BD6882309F4F5
:102A1000CACE812C82E0982EA80CB91CEF81F885D3
:102A200080899189A289B389880D991DA11DB11D45
:102A3000808B918BA28BB38BE818F908F8CE20E03D
:102A4000CF018096E1D6009709F4ADCE20E032E0C8
:102A50002C193D0947012E153F0508F44901BC0119
:102A60006C0D7D1DA401C5010E945242D5CFCF013E
:102A700080964B835C836D837E8383D64B815C81A0
:102A80006D817E8181116CCF8ECE28960FB6F89421
:102A9000DEBF0FBECDBFDF91CF911F910F91FF9091
:102AA000EF90DF90CF90BF90AF909F908F907F90EE
:102AB0006F905F904F903F900895FF920F931F93F8
:102AC000CF93DF931F92CDB7DEB78C01FC018089D5
:102AD0009189A289B3899C01AD0175E0569547950E
:102AE000379527957A95D1F7F22FFF70FF2E11F0C9
:102AF000611115C041E050E0BE016F5F7F4FC8011A
:102B000010DE813019F080E090E01AC0F801808971
:102B10009189A289B3894F96A11DB11D04C08096E9
:102B2000A11DB11DF801808B918BA28BB38BF80195
:102B3000868197818796F0E2FF9E800D911D11247A
:102B40000F90DF91CF911F910F91FF900895FC019D
:102B50008081811114C080E2DF01982F1D929A9527
:102B6000E9F777836683DB0115969C91903119F024
:102B7000903229F480E4808381E08283089580E0AC
:102B800008956F927F928F929F92AF92BF92CF9251
:102B9000DF92EF92FF920F931F93CF93DF9300D0BA
:102BA0001F92CDB7DEB77C01722E80E2D7011D9255
:102BB0008A95E9F7FB01C680D780D7011796DC928A
:102BC000CE92169715965C934E931497848D958D9F
:102BD000A68DB78DF70180879187A287B3874F7045
:102BE0005527D601979695E0440F551F9A95E1F722
:102BF000A40FB51F1B968C911B9783FF04C0D701B0
:102C00001C9280E094C0F601E40FF51F82A9877141
:102C1000F70180831B969C91987111F488608083E2
:102C2000D70113960C931397872D827319F08C910B
:102C3000817129F7872D8F70F7018283F60183A1B7
:102C400094A1A5A1B6A1F701848B958BA68BB78B18
:102C5000F601E40FF51F83AC94ACA12CB12CB401A8
:102C6000552744279F012F5B3F4FD9018D909C90A2
:102C7000A12CB12C842A952AA62AB72A74FE31C029
:102C800081149104A104B10409F44BC09E012F5F8B
:102C90003F4FB501A401C60165D6682E87FDAFCFB1
:102CA00000E010E09801B501A401C601EBD588232E
:102CB00009F4A5CFF6014085518562857385841698
:102CC0009506A606B70620F480869186A286B3866E
:102CD00089809A80AB80BC806110D8CF811121C0DF
:102CE0008ECFD7015C968D929D92AD92BC925F97EC
:102CF000ED5BFF4F80819181A281B381F701808FCD
:102D0000918FA28FB38F75FE11C0D70158964D9148
:102D10005D916D917C915B97C7013FDC811106C08D
:102D20006ECFF701828180688283EDCF81E00F90C2
:102D30000F900F900F90DF91CF911F910F91FF9007
:102D4000EF90DF90CF90BF90AF909F908F907F904B
:102D50006F900895CF93DF93EC01262F4C895D8906
:102D60006E897F898E819F8180964ED5009761F014
:102D70002C813D812F70332745E0220F331F4A9568
:102D8000E1F7820F931F02C080E090E0DF91CF91C6
:102D90000895CF93DF93FC012081211102C081E0CF
:102DA0002FC0EC01828187FF24C061E0CF01D2DF18
:102DB000FC01892B29F489818160898380E020C00E
:102DC0008081853EC1F3888183FF08C0888D998DFD
:102DD000AA8DBB8D848F958FA68FB78F8C8D9D8D7F
:102DE000AE8DBF8D938F828FB58BA48B8A818F77A9
:102DF0008A838E819F818096C4D48823E1F2CFCFCD
:102E0000DF91CF9108952F923F924F925F926F92F0
:102E10007F928F929F92AF92BF92CF92DF92EF926A
:102E2000FF920F931F93CF93DF93CDB7DEB72A970F
:102E30000FB6F894DEBF0FBECDBF9E838D833B01DE
:102E40005A834983DC018C9183FF10C012968C91C8
:102E500081FF0CC082FF12C0ED81FE81408D518D3B
:102E6000628D738DCF0199DB811108C0ED81FE81E8
:102E70008181816081838FEF9FEFB3C189819A81C6
:102E8000AC0160E070E0ED81FE8180899189A289CA
:102E9000B38980959095A095B09584179507A6075E
:102EA000B70720F3C980DA803C96FC83EB832224A9
:102EB0002A94322C2101AD81BE8150964D915D91B5
:102EC0006D917C915397C114D10409F461C1AD8116
:102ED000BE8116968D919C9117978A019B0169E09E
:102EE00036952795179507956A95D1F7DC011396C6
:102EF000EC91BE2EB0227A01B1E0FB22B1103DC0B0
:102F0000E114F104D1F5ED81FE8144855585668596
:102F10007785411551056105710571F02B813C8163
:102F200021D587FDA3CF811128C08D819E810E946C
:102F30000321811122C09ACFED81FE81848D958D70
:102F4000A68DB78D0097A105B10589F4CF010E9428
:102F50000321882309F48ACFED81FE81848595853C
:102F6000A685B785848F958FA68FB78F06C0ED8114
:102F7000FE8184879587A687B787AD81BE81169627
:102F8000ED91FC9117971C964D915D916D917C91FF
:102F90001F974250510961097109048004C0440F10
:102FA000551F661F771F0A94D2F780899189A289DD
:102FB000B389480F591F6A1F7B1F4B0D511D611D9F
:102FC000711DE114F10429F4C114B2E0DB0608F02C
:102FD0003EC080E092E08E199F0986018C159D0508
:102FE00008F48C01E114F104A9F4AD81BE8150967E
:102FF0008D909D90AD90BC90539758968D919D91DA
:103000000D90BC91A02D88169906AA06BB0610F05B
:1030100025E001C021E0CF018096F6D3009709F4A6
:1030200025CFA801B3018E0D9F1D0E945242E00ED4
:10303000F11EE114B2E0FB0609F097C0ED81FE81BC
:103040008681978180969DD381118FC00FCF03A178
:1030500014A125A136A1C11484E0D80608F46BC0E0
:1030600082818B1990E0AD2CA694B12C8A159B051A
:1030700008F45C01041715072607370760F0D9012B
:10308000C8018A0D9B1DA11DB11D481759076A076C
:103090007B0708F4A0C0AD81BE811696ED91FC912E
:1030A0001797E080F180F7018581833039F099E04E
:1030B000440F551F661F771F9A95D1F79A01AB01F0
:1030C00069E1C701E7D2811104C0430100E010E0CB
:1030D0000FC083E3D7018C9315C0A4016CEFC70127
:1030E0000E94910D882371F00F5F1F4FFEEF9F1A12
:1030F0000A151B0559F00E94062C8111EECF8AE5B6
:10310000F7018083C7010E947E0D11C00E94062C2A
:10311000882351F0102F0027110F8DEF0E94720DA0
:10312000C7010E947E0D21C086E5D7018C93C7019F
:103130000E947E0D9BCE041715072607370729F43A
:1031400010A223A234A245A256A2AD81BE8116963A
:10315000ED91FC9117979301808191810E94C20D9E
:10316000882309F483CE00E012E0ED81FE8180899E
:103170009189A289B389800F911FA11DB11D808BF8
:10318000918BA28BB38B600E711EC01AD10A93CEA5
:1031900058968D919D910D90BC91A02D8417950707
:1031A000A607B70748F4ED81FE81408F518F628FEB
:1031B000738F828180688283AD81BE8112968C91EB
:1031C00083FD03C089819A810CC08D819E81E1DDE0
:1031D0008111F8CF4BCE10A223A234A245A256A251
:1031E0005ACF2A960FB6F894DEBF0FBECDBFDF913F
:1031F000CF911F910F91FF90EF90DF90CF90BF90F4
:10320000AF909F908F907F906F905F904F903F9086
:103210002F900895CF93DF93EC01BBDD1882DF91EF
:10322000CF910895CF92DF92EF92FF920F931F9369
:10323000CF93DF93CDB7DEB7E3970FB6F894DEBF39
:103240000FBECDBF7C018B015BAB4AABD22E198286
:103250001A82FC018081882311F080E053C0FB01B9
:1032600080818077D1F3EAA9FBA980818F32C9F4EC
:10327000EAA9FBA980818F3221F43196FBABEAAB3E
:10328000F7CFF80166817781811103C0C7015FDC48
:1032900039C0CE0101965BDC8823F9F28E010F5F05
:1032A0001F4F80E2C82EAE014E5C5F4FBE016F5DC6
:1032B0007F4F8AA99BA9E8D3882379F2EAA9FBA9C1
:1032C00080818823C1F021E0AE014F5D5F4FB801DE
:1032D000C7010BD5882309F4C0CFF701DE01119691
:1032E0008C2D01900D928A95E1F7C70193DF8E0135
:1032F0000F5F1F4FD8CF2D2DAE014F5D5F4FB8012F
:10330000C701F3D4E3960FB6F894DEBF0FBECDBF6E
:10331000DF91CF911F910F91FF90EF90DF90CF90B1
:1033200008958F929F92AF92BF92EF92FF920F9368
:103330001F93CF93DF93EC01888185FF02C010E0DB
:1033400066C088899989AA89BB8981159E4FAF413A
:10335000B105A8F7CE0157D7182F882381F3EE8146
:10336000FF814C855D856E857F85425051096109DD
:103370007109048004C0440F551F661F771F0A940B
:10338000D2F780889188A288B388840E951EA61EE5
:10339000B71E25E0B501A401CF01809635D27C018E
:1033A000892B69F280E092E0F7019C011192215093
:1033B0003040E1F701E0EE81FF819281091780F44E
:1033C0009701B501A401400F511D611D711D808140
:1033D00091810E94C20D882309F4B1CF0F5FEBCF1A
:1033E000492F50E060E070E089E0440F551F661FF0
:1033F000771F8A95D1F788899989AA89BB89480F4F
:10340000591F6A1F7B1F488B598B6A8B7B8B812FBF
:10341000DF91CF911F910F91FF90EF90BF90AF90F0
:103420009F908F900895AF92BF92CF92DF92EF92CC
:10343000FF920F931F93CF93DF93CDB7DEB7A09783
:103440000FB6F894DEBF0FBECDBF8C01DB019C919F
:10345000907709F4A2C07B0123ECC80146D48823ED
:1034600009F49BC081E0F801828380E1D82ED082EC
:10347000C80157DF882309F490C0F8018485958539
:10348000A685B785848F958FA68FB78F40E050E0D3
:10349000BA01C80182D8C8017CDC882309F47DC048
:1034A00061E0C80157DC009709F477C0DC011B9686
:1034B000DC9220E2FC01DE01119601900D922A952A
:1034C000E1F7FC01A488B588C28CD38C8EE2898395
:1034D000FE013296CE010C9620E22193E817F907FF
:1034E000E1F7D8011696ED91FC9117975C964D91F6
:1034F0005D916D917C915F9742505109610971090D
:10350000048004C0440F551F661F771F0A94D2F72A
:1035100080899189A289B389480F591F6A1F7B1F2F
:1035200021E0CF01809670D10097B9F1BE8AAD8AB3
:10353000DC8ECB8E20E2FE013196DC0101900D92F3
:103540002A95E1F72EE22A83F701448D558D668D89
:10355000778D7E8B6D8B5C8F4B8F20E2FE013196D9
:10356000DC01909601900D922A95E1F7D80116960C
:103570008D919C9117978096A0960FB6F894DEBF18
:103580000FBECDBFDF91CF911F910F91FF90EF90B4
:10359000DF90CF90BF90AF90F4C080E0A0960FB6C0
:1035A000F894DEBF0FBECDBFDF91CF911F910F9179
:1035B000FF90EF90DF90CF90BF90AF900895CF93A2
:1035C000DF93FC012381211110C0EC010180F28105
:1035D000E02D908181819CBD8DBDE981FA8160E003
:1035E00082810E946B0A81E08B83DF91CF910895E5
:1035F000CF92DF92EF92FF920F931F93CF93DF93BF
:103600008C017B01EA010E945C0B6B010E94770D2B
:10361000F80184838F3F51F40E945C0B6C197D0983
:103620006D32714098F385E5F80103C08E3F39F0A3
:1036300080E58083C8010E947E0D80E022C0209733
:10364000C9F021978FEF8EBDF7012FEFCF018E19B3
:103650009F098C179D0738F40DB407FEFDCF8EB57A
:103660002EBD8193F3CF0DB407FEFDCF8EB5CE0DE9
:10367000DF1D8883F80114820E94770D0E94770D68
:1036800081E0DF91CF911F910F91FF90EF90DF903C
:10369000CF900895EF92FF921F93CF93DF9300D0C6
:1036A0001F92CDB7DEB77C01162F29833A834B8357
:1036B0005C83FC018381811102C0C70180DF0E940D
:1036C000062C812F80640E94720D8C810E94720DE5
:1036D0008B810E94720D8A810E94720D89810E94E5
:1036E000720D112311F087E801C085E90E94720D67
:1036F0001C3011F40E94770D10E00E94770DF70145
:10370000848387FF04C01F3F11F01F5FF6CF0F9027
:103710000F900F900F90DF91CF911F91FF90EF903E
:1037200008950F931F93CF93DF93EC0189018D814F
:10373000833039F089E0440F551F661F771F8A9543
:10374000D1F79A01AB0161E1CE01A4DF882319F022
:1037500080E388830CC040E052E0B801CE0148DF2E
:10376000182F882321F0CE010E947E0D04C0CE01C7
:103770000E947E0D10E0812FDF91CF911F910F915C
:103780000895EF92FF921F93CF93DF93FC01208166
:1037900020FF32C0EC017C01F7E0EF0EF11C4B8101
:1037A0005C816D817E81E981FA81970180819181BF
:1037B0000E94C20D182F811102C010E01EC0888126
:1037C00081FD04C088818E7F888317C0E981FA81DA
:1037D00044855585668577858B819C81AD81BE81C9
:1037E000480F591F6A1F7B1F9701808191810E949A
:1037F000C20D8111E7CFE1CF11E0812FDF91CF9191
:103800001F91FF90EF900895CF92DF92EF92FF9279
:103810001F93CF93DF93EC016A017B01122F8B8101
:103820009C81AD81BE8184179507A607B707E1F09B
:10383000CE01A7DF811103C080E090E01BC012FF22
:1038400006C01882CB82DC82ED82FE820DC0E98147
:10385000FA819E01295F3F4FB701A60180819181C6
:1038600060DF8111EECFE8CF13708881182B1883A9
:10387000CE010796DF91CF911F91FF90EF90DF90DF
:10388000CF9008958F929F92AF92BF92CF92DF9286
:10389000EF92FF920F931F936A017B014801590138
:1038A000423051056105710510F480E050C0FC0103
:1038B000408D518D628D738D4C155D056E057F05B4
:1038C000A0F32581203239F54489558966897789A5
:1038D00097018601E7E03695279517950795EA95B4
:1038E000D1F7400F511F621F731F23E080968CDFBA
:1038F0000097D9F2E894C7F8DD24EE24FF24CC0C1D
:10390000DD1CCC0CDD1CFC01EC0DFD1D80829182C8
:10391000A282B3821BC0203141F6FC014489558943
:10392000668977894D0D511D611D711D23E08096BB
:103930006BDF009709F4B9CFDD24EE24FF24CC0C13
:10394000DD1CFC01EC0DFD1D9182808281E01F9148
:103950000F91FF90EF90DF90CF90BF90AF909F902E
:103960008F900895CF92DF92EF92FF920F931F9363
:10397000CF93DF93EC016A017B018901423051054D
:103980006105710510F48FEF61C0888D998DAA8D46
:10399000BB8D84179507A607B707A8F38D818032E2
:1039A00039F58C899D89AE89BF89E7E07695679561
:1039B00057954795EA95D1F7480F591F6A1F7B1F06
:1039C00022E0CE01809620DF0097E9F2E894C7F864
:1039D000DD24EE24FF24CC0CDD1CCC0CDD1CFC0112
:1039E000EC0DFD1D80819181A281B381BF701DC04E
:1039F000803149F64C895D896E897F894D0D511D55
:103A0000611D711D22E0CE018096FEDE009709F453
:103A1000BACFDD24EE24FF24CC0CDD1CFC01EC0D20
:103A2000FD1D80819181A0E0B0E0488D598D6A8DA7
:103A30007B8D481759076A077B0738F0F8018083A8
:103A40009183A283B38381E001C080E0DF91CF91B5
:103A50001F910F91FF90EF90DF90CF900895611527
:103A6000710579F0FB0101900020E9F73197AF0172
:103A7000461B570BDC01ED91FC910280F381E02D98
:103A8000199480E090E00895AF92BF92CF92DF92B8
:103A9000EF92FF920F931F93CF93DF93FB01DC0113
:103AA00001962C912032D9F3B483A3839D0189011F
:103AB0000A1B1B0BE90189919E018823C1F08F32FB
:103AC000B1F08C3511F480E0F2C0982F977F9232DC
:103AD000D1F38A33C1F3982F9F7B9C33A1F392ECEF
:103AE000980F923080F380528F3508F3ECCF0A0F95
:103AF0001B1FC801682F392FEC012991CE012032FC
:103B0000C9F32F32B9F3EA016883398398012A1B7C
:103B10003B0B0A171B0741F0E8018A918E018E3298
:103B2000A9F3803299F303C0A12CB12C05C059012F
:103B30002F3F310509F03CF6B282A182CF010696F3
:103B40009F012F5E3F4F40E2EC014993CE01C21727
:103B5000D307D1F7CD01AC014A1B5B0BEC013991C6
:103B6000CE013E32C1F33032B1F39A0191E0452BE0
:103B700009F090E0A5014150510938F0BD01640FF2
:103B8000751FEB0188818E32B1F717E060E000E02D
:103B900070E088E0E82E2A153B050CF06CC06D0142
:103BA000C20ED31EE6018881803209F45BC08E32DA
:103BB00029F44217530709F055C004C08232E1F0DE
:103BC0008C37D1F0D6EDFD2EF80ED5E0DF1510F0D4
:103BD0008D3291F4C6ECFC2EF80EC5E0CF1560F4E2
:103BE000D5EAFD2EF80ED2E0DF1530F4CFEDFC2E35
:103BF000F80ECDE5CF1520F42417350781F438C031
:103C000024173507A9F1161718F1F82ECFE9DC2E85
:103C1000D80ED9E1DD1548F080527E290CC0161768
:103C2000B8F090E08FE5CFE5FC2ECFEBFC0ED9E1AC
:103C3000DF1508F00E29FF24F394F60E6F01C60E6F
:103C4000D11CE6018E83D6E0DF1570F0F5820CC042
:103C50001A3081F0421753076CF09A011AE068E0BD
:103C6000D0E1ED2E90E001C06F2D2F5F3F4F93CF3D
:103C70001A30B9F490E08681803209F424CF992378
:103C800029F0072309F072E0708309C081E0808386
:103C90008581E80FF11D8EE7868381E3878381E0CC
:103CA00006C09A011AE068E0D0E1ED2EDECFDF9188
:103CB000CF911F910F91FF90EF90DF90CF90BF9029
:103CC000AF900895FC01AC01455F5F4F80E090E844
:103CD000899F90011124982F9695922B2191892FDD
:103CE000820FE417F50799F708952F923F924F92AC
:103CF0005F926F927F928F929F92AF92BF92CF927C
:103D0000DF92EF92FF920F931F93CF93DF93CDB784
:103D1000DEB72A970FB6F894DEBF0FBECDBF4C01B9
:103D20008B01FA01A180B280DB018C91807711F4C4
:103D300080E050C2D4018C918111FACF90819370B0
:103D400009F43CC2C5010C966DE070E00E9412427D
:103D500077247394760E2A837F011A87098740E0BF
:103D600050E0BA01C8010E94CD121C821D82198246
:103D7000612C10E000E01B8297012A5F3F4F3F83D8
:103D80002E83E985FA8580899189A289B3891C01EE
:103D90002D01A5E05694479437942794AA95D1F71E
:103DA000610161E0CF010E945D15009741F4A98592
:103DB000BA8511968C91882309F497C0B9CFFC017C
:103DC0002081253E11F021110AC0111102C02C8260
:103DD0003D82171508F41F5F211105C086C0171515
:103DE00008F4EFC102C0253EF1F12E32E1F1DC0111
:103DF0001B963C911B973F3009F057C0011109C039
:103E000026FFBFCF022F0F711D962C912983602EA4
:103E100009C06A94261127C0DC011D962C913981B6
:103E2000321321C0462D50E0415051096DE0649F8E
:103E30009001659F300D11242A153B05A0F4FC016B
:103E400060E0653018F48181928107C06B3018F40E
:103E50008481958102C0868197812A153B0529F4CA
:103E6000892B09F48ECF00E08CCF8F3F910509F0AC
:103E7000D0F74FEB480F4A3110F0782F02C070E2B4
:103E8000780FA9014F5F5F4FD70113968D919C91D9
:103E90001497DC01A20FB31F8C919FEB980F9A31FE
:103EA00008F4805E7813DFCF8EC133FDDCCF0023B2
:103EB00041F0B1E06B123CCF05DF2981821338CF8E
:103EC00010C04BE050E06E817F810E944542892BFB
:103ED00009F057CFD7018C9180FF03C031E03B83BD
:103EE00050CF2A8127FF62C123CF8A818274823416
:103EF00009F01ECF112359F0CC80DD8008C060E0AE
:103F000089859A850E945D15892B21F01F5F171501
:103F1000B0F317C0A985BA8511968C91882389F0D2
:103F200007CF89859A85FDD9882309F401CFA98512
:103F3000BA851696ED91FC9117978281823018F41C
:103F4000105F171570F32B81222309F473C0D7017A
:103F500015966C9002E010E07EE7372E2701B6E060
:103F60004B0E511C41C0F3E0F61510F453E0652EE2
:103F700034E0360D282F2F70E32FF0E02A3008F0C0
:103F800051C0205DEE0DFF1D268344E09695879578
:103F90004A95E1F73150631668F3F701E60DF11D1C
:103FA000368240E050E0BA0189859A850E94CD12A0
:103FB00061E089859A850E945D150097A9F1FC0151
:103FC00020812223B9F1238523FDF2CF4BE050E07D
:103FD000BC01C2010E944542892B51F70F5F1F4F60
:103FE0000436110509F4A4CEF70141815281C801BC
:103FF000840F951F0380F481E02D4E0F5F1FE4179F
:10400000F50709F4B0CF9C0165E0220F331F6A95D4
:10401000E1F7820F931F2191022E000C330B8227B0
:104020009327EDCF295CAECFA985BA8511968C91E7
:1040300081117ECEA60160E070E035E0440F551F8F
:10404000661F771F3A95D1F789859A850E94CD1210
:10405000882309F46DCE0FEF070D102F9FE0492E36
:104060006701F6E0CF0ED11C2DE0522E112309F48A
:104070005DC060E089859A850E945D153C01892BB1
:1040800009F456CEA985BA851696ED91FC9117973D
:1040900080A1816080A3212F101301C02064F3014F
:1040A000208343861486C60128870CDED3011D9623
:1040B0008C931D975B961C921E925A97F701438131
:1040C000548128852F71822F90E00197589E90018E
:1040D000599E300D1124F30160E02A153B0540F490
:1040E000DA01A20FB31F8C91082E000C990B0AC0A5
:1040F00081E090E02A153B0511F480E090E0919575
:1041000081959109653018F49283818307C06B30E3
:1041100018F49583848302C0978386836F5F2F5F33
:104120003F4F32966D30C9F61150A0CFA985BA85A0
:1041300050964D915D916D917C91539785E0769568
:104140006795579547958A95D1F76A0160E0CD014B
:104150000E945D15009709F4EBCD20E2FC0111925D
:104160002A95E9F7F70136962BE0DC0101900D92D4
:104170002A95E1F7D7012C912871FC01248721E2CF
:1041800038E2318B208B40E058E057874687338BED
:10419000228B318F208F578B468BA985BA85169637
:1041A000ED91FC91179780A1816080A32A81A601DF
:1041B00069857A85C4010E94C1150CC07724739467
:1041C000CACD10E012CE6F5F32966D3009F4D9CDB2
:1041D0009A0137CE2A960FB6F894DEBF0FBECDBF38
:1041E000DF91CF911F910F91FF90EF90DF90CF90D3
:1041F000BF90AF909F908F907F906F905F904F9007
:104200003F902F9008953F924F925F926F927F92CE
:104210008F929F92AF92BF92CF92DF92EF92FF92D6
:104220000F931F93CF93DF93CDB7DEB728970FB6C9
:10423000F894DEBF0FBECDBF4C01DC0112968C910D
:104240001297806812968C9312971C964D905D90F1
:104250006D907C901F971696AD90BC901797411467
:1042600051046104710461F4D50118968D919D91FA
:104270000D90BC91A02D8D839E83AF83B88704C021
:104280004D825E826F827886CD80DE80EF80F884FA
:10429000BFEFCB1ADB0AEB0AFB0AF501808D918D8B
:1042A000A28DB38D8C159D05AE05BF0528F482E067
:1042B000C82ED12CE12CF12C9E012F5F3F4FB7016E
:1042C000A601C5014FDB87FD1FC0882341F089810E
:1042D0009A81AB81BC81892B8A2B8B2B51F08D81EC
:1042E0009E81AF81B885C816D906EA06FB0681F61D
:1042F0000BC00FEF1FEF2FEF3FE0B701A601C50185
:10430000C1DA382E811102C0312C1AC04114510477
:104310006104710449F097018601B301A201C5014E
:10432000B1DA811108C0F0CFD5011896CD92DD9297
:10433000ED92FC921B97F401C486D586E686F7863B
:10434000832D28960FB6F894DEBF0FBECDBFDF9148
:10435000CF911F910F91FF90EF90DF90CF90BF9082
:10436000AF909F908F907F906F905F904F903F9015
:104370000895CF92DF92EF92FF92CF93DF93EC01FB
:10438000219680EFC82E8EEFD82EEE24EA94FE2CD4
:10439000C701B6010E94320FFE01319780839883D6
:1043A0008FEFC81AD80AE80AF80A229687EFC816CB
:1043B0008EEFD8068FEFE806F80651F78EE0DF9112
:1043C000CF91FF90EF90DF90CF900895CF93DF9340
:1043D00061E08FE30E94E80A61E084E00E94E80A5D
:1043E00061E083E10E94E80A61E081E10E94E80A5D
:1043F00061E082E00E94E80A61E08CE30E94E80A42
:1044000061E080E30E94E80A61E08CE20E94E80A31
:1044100061E08AE30E94E80A61E083E00E94E80A22
:1044200061E080E10E94E80A61E082E10E94E80A1E
:1044300061E085E00E94E80A61E08EE30E94E80AFC
:1044400061E080E40E94E80A61E082E40E94E80AF8
:1044500061E083E40E94E80A61E088E20E94E80AE1
:1044600061E084E20E94E80A61E08EE20E94E80ACC
:1044700061E08AE20E94E80A61E086E20E94E80ABE
:1044800061E082E20E94E80A80E00E948D2E61E0F5
:1044900086E10E94E80A109A61E088E10E94E80A39
:1044A000129A61E08AE10E94E80A149A61E08CE1C4
:1044B0000E94E80A169A61E08EE10E94E80A479A93
:1044C00061E080E20E94E80A459A61E085E40E948A
:1044D000E80AC8E0D1E088818068888361E084E4EC
:1044E0000E94E80A88818064888361E081E40E94F8
:1044F000E80A88818860888362E089E30E94E80A8C
:10450000888180648883888180688883149A888100
:1045100088608883169A64EF71E080E090E00E94E2
:10452000240B0E94BF100E94970F0E94BF108EE5BF
:104530009EE00E94522F68EE73E080E090E0DF91F1
:10454000CF910C94240B8F929F92AF92BF92CF92F7
:10455000DF92EF92FF920F931F93CF93DF938BE441
:104560009EE00E94312F8DEF93E00E949A1261E04D
:104570008FEF97E00E941C2C882309F4F6C08091ED
:104580005E0B90915F0BA091600BB091610B8093DB
:104590005C0490935D04A0935E04B0935F0440912B
:1045A0004A0250914B0260914C0270914D024817A3
:1045B00059076A077B0720F48DE29EE00E94522F84
:1045C0001092E1071092E2071092E3071092E407BD
:1045D000C12CD12C760180915C0490915D04A09156
:1045E0005E04B0915F04B695A79597958795C81618
:1045F000D906EA06FB0608F0A7C040E850E060E6EE
:1046000074E086E49BE00E9491134601570100E0AC
:1046100010E0F801E05AFB4FC181D0E0DC2FCC273D
:104620008081C82BC501B4010E94320F8C179D07F1
:1046300009F44DC08091E1079091E207A091E30752
:10464000B091E4070196A11DB11D8093E1079093FD
:10465000E207A093E307B093E40782E09EE00E94A4
:10466000522F84EF9DE00E94312F40E150E0C701BE
:10467000B601A0D38CEE9DE00E94312FC501B4019C
:104680000E94320FAC0160E070E020E189E99AE01D
:104690000E94BA0966E073E089E99AE0E0D980EE09
:1046A0009DE00E94312FAE0160E070E020E189E9D9
:1046B0009AE00E94BA0966E073E089E99AE0CFD9EE
:1046C00086E49BE00E940A1967E074E04BC00E5F2D
:1046D0001F4F8FEF881A980AA80AB80A00381105E8
:1046E00009F097CFD701C6019F70AA27BB27892B56
:1046F0008A2B8B2B19F5A4E6B0E0A70196010E9446
:10470000BD3F00915C0410915D0420915E043091E6
:104710005F043695279517950795A90198012054B0
:104720003109410951090E94A13F822F0E9445127F
:104730006AE973E089E99AE00E940A0A80E4C80EF7
:10474000D11CE11CF11C47CF88E093E00E94612F4F
:104750008BEC9DE00E94522F86E49BE00E940A1998
:104760006BE174E08FE094E008C086E19EE00E9477
:10477000522F63E274E08AE294E0DF91CF911F91BF
:104780000F91FF90EF90DF90CF90BF90AF909F90F0
:104790008F900C9452118F929F92AF92BF92CF92B2
:1047A000DF92EF92FF920F931F93CF93DF938EE7E9
:1047B00093E00E949A1285EE97E09F938F938FEF7C
:1047C00097E09F938F932AE833E03F932F939F9333
:1047D0008F930E9476428BEB9DE00E94312F8FEFEA
:1047E00097E00E94612F8AEA9DE00E94312F61E0EC
:1047F0008FEF97E00E941C2C2DB73EB7285F3F4FEC
:104800000FB6F8943EBF0FBE2DBF882309F4DEC05B
:1048100080915E0B90915F0BA091600BB091610B4A
:1048200080935C0490935D04A0935E04B0935F0456
:1048300040914A0250914B0260914C0270914D029E
:1048400084179507A607B70721F085E89DE00E9429
:10485000522F0E94220EC12CD12C7601CBE3D6E040
:1048600080915C0490915D04A0915E04B0915F041E
:10487000B695A79597958795C816D906EA06FB06BB
:1048800008F084C040E052E060E674E086E49BE01B
:104890000E9491134AEA50E065E575E080E090E0FF
:1048A0000E94700F45E550E06AEA72E080E090E017
:1048B0000E94700F43E350E0C701B6010E94700FE1
:1048C0004091610450E0542F442780916004482BAC
:1048D000C701B6010E94700F460157013FEF831ACE
:1048E000930AA30AB30A02E010E0F801E05AFB4F72
:1048F000418150E0542F44278081482BC501B401E9
:104900000E94700F0E5F1F4F8FEF881A980AA80A37
:10491000B80A011522E0120741F749E250E0C70149
:10492000B6010E94700FCE010197F1F7D701C601C1
:104930009F70AA27BB27892B8A2B8B2B11F5A4E606
:10494000B0E0A70196010E94BD3F00915C04109168
:104950005D0420915E0430915F043695279517958C
:104960000795A90198013150410951090E94A13FC1
:10497000822F0E9445126AE973E089E99AE00E9459
:104980000A0A3FEFD31AE30AF30A6ACF88E093E0FA
:104990000E94612F87E59DE00E94522F63E173E042
:1049A0008EE793E00E9452110E941F0E86E49BE066
:1049B000DF91CF911F910F91FF90EF90DF90CF90FB
:1049C000BF90AF909F908F900C940A198EE69DE057
:1049D000DF91CF911F910F91FF90EF90DF90CF90DB
:1049E000BF90AF909F908F900C94522F8F929F9278
:1049F000AF92BF92CF92DF92EF92FF921F93CF932D
:104A0000DF938EE793E00E949A1285EE97E09F93E2
:104A10008F938FEF97E09F938F932AE833E03F9334
:104A20002F939F938F930E94764283ED9CE00E9488
:104A3000312F8FEF97E00E94612F88EB9CE00E945E
:104A4000312F61E08FEF97E0F7D62DB73EB7285FA3
:104A50003F4F0FB6F8943EBF0FBE2DBF882309F419
:104A6000DAC080915E0B90915F0BA091600BB091CA
:104A7000610B80935C0490935D04A0935E04B093FB
:104A80005F0440914A0250914B0260914C02709138
:104A90004D0284179507A607B70721F083E99CE02C
:104AA0000E94522F0E94220EC12CD12C760110E0C0
:104AB00080915C0490915D04A0915E04B0915F04CC
:104AC000B695A79597958795C816D906EA06FB0669
:104AD00008F082C040E850E060E674E086E49BE0C5
:104AE0000E949113809160068130C1F44AEA50E03F
:104AF00065E575E580E090E00E94700F45E550E0C7
:104B00006AEA7AE280E090E00E94700F40EA50E0AA
:104B100065E575E580E090E00E94700F4601570161
:104B2000C0E0D0E0FE01E05AFB4F418150E0542F3D
:104B300044278081482BC501B4010E94700F229642
:104B40003FEF831A930AA30AB30AC038D10551F77D
:104B500080916006813019F40E94590F182F8091BE
:104B60006006813039F414FF05C089E69CE00E949C
:104B7000522F40C0D701C6019F70AA27BB27892B9F
:104B80008A2B8B2B19F5A4E6B0E0A70196010E94B1
:104B9000BD3F80905C0490905D04A0905E04B09056
:104BA0005F04B694A79497948794A5019401205428
:104BB0003109410951090E94A13F822F0E944512EB
:104BC0006AE973E089E99AE00E940A0A80E4C80E63
:104BD000D11CE11CF11C6CCF88E093E00E94612F96
:104BE00082E59CE00E94522F63E173E08EE793E040
:104BF0000E9452110E941F0E86E49BE0DF91CF912C
:104C00001F91FF90EF90DF90CF90BF90AF909F905B
:104C10008F900C940A198CE79CE0DF91CF911F9143
:104C2000FF90EF90DF90CF90BF90AF909F908F90CC
:104C30000C94522F8F929F92AF92BF92CF92DF929D
:104C4000EF92FF920F931F9386E49CE00E94522FF5
:104C500087E39CE00E94312F82E394E00E949A1245
:104C600081E090E0A0E0B0E08093E1079093E2075C
:104C7000A093E307B093E407C12CD12C7601809177
:104C80004A0290914B02A0914C02B0914D02B69510
:104C9000A79597958795C816D906EA06FB0608F0EA
:104CA00048C0C701B6010E94320F80904A0290901E
:104CB0004B02A0904C02B0904D02019671F075012C
:104CC0006401F694E794D794C7941092E107109288
:104CD000E2071092E3071092E407D701C6019F7024
:104CE000AA27BB27892B8A2B8B2BE9F4A4E6B0E0FB
:104CF000A70196010E94BD3F950184013695279535
:104D000017950795A90198012250310941095109C8
:104D10000E94A13F822F0E9445126AE973E089E94F
:104D20009AE00E940A0A8FEFC81AD80AE80AF80A1D
:104D3000A6CF8091E1079091E207A091E307B0919F
:104D4000E407892B8A2B8B2B59F088E093E00E9493
:104D5000612F83E29CE00E94522F6BE174E006C059
:104D600082E19CE00E94522F67E074E082E394E0CD
:104D70001F910F91FF90EF90DF90CF90BF90AF9079
:104D80009F908F900C945211CF93DF93AC01990FA9
:104D9000660B770B89E99AE00E94742FEC0166E0BC
:104DA00073E089E99AE00E942F1D8C0F9D1FDF910F
:104DB000CF910895CF93DF934115510559F4E091B8
:104DC000990AF0919A0A0190F081E02D89E99AE020
:104DD000199507C0242FAB01BC0189E99AE00E9414
:104DE000BA09EC0166E073E089E99AE00E942F1DA0
:104DF0008C0F9D1FDF91CF9108954F925F926F921C
:104E00007F928F929F92AF92BF92CF92DF92EF925A
:104E1000FF926B017C01B42E9B01AC010E940E42FB
:104E2000882319F06EE374E027C026013701E89467
:104E300077F82FEF3FEF4FE75FE7C301B2010E9422
:104E40000E4281110DC02FEF3FEF4FE75FE7C30127
:104E5000B2010E945D4018161CF462E474E00CC0BC
:104E60002FEF3FEF4FE75FE4C701B6010E94A74174
:104E7000181694F466E474E089E99AE0FF90EF90E4
:104E8000DF90CF90BF90AF909F908F907F906F906A
:104E90005F904F900C942F1D2FEF3FEF4FE75FEC8B
:104EA000C701B6010E945D4087FDE4CF20E030E0FD
:104EB000A901C701B6010E945D4087FF0BC06DE2EA
:104EC00089E99AE00E94030A4C01F7FAF094F7F896
:104ED000F09402C0812C912CA12C60E070E080E065
:104EE0009FE3AB1441F020E030E040E251E40E9447
:104EF0006140A394F6CF9B01AC01C701B6010E94AB
:104F0000F93F2B013C010E94C9406B017C010E94CA
:104F1000F5409B01AC01C301B2010E94F83F2B0197
:104F20003C012AE0B701A60189E99AE00E94BA098A
:104F30007C01E80CF91CBB2039F06EE289E99AE0AB
:104F40000E94030AE80EF91EDB2CDD2031F120E07F
:104F500030E040E251E4C301B2010E94AB412B01B9
:104F60003C010E94C9404B01A12CB12C2AE0B501A3
:104F7000A40189E99AE00E94BA09E80EF91EC50168
:104F8000B4010E94F5409B01AC01C301B2010E9433
:104F9000F83F2B013C01DA94D8CFC701FF90EF9086
:104FA000DF90CF90BF90AF909F908F907F906F9049
:104FB0005F904F900895CF93DF931092370810922F
:104FC000360810923508109234081092330881E0A8
:104FD000809332081092310861E084E10E946B0AEC
:104FE00061E085E10E946B0A8091B9008E7F809319
:104FF000B9008091B9008D7F8093B90088E48093D7
:10500000B80085E48093BC001092BB0D8091C00D68
:10501000823018F098E09093BB0D8093BE0D62E350
:1050200070E080E090E00E94240B6091C10D86EB5F
:105030009DE00E94E30C68EE73E080E090E00E9447
:10504000240B60E386EB9DE00E94470DCBE4D6E4A1
:10505000CE010197F1F760E386EB9DE00E94470DDA
:105060002197F1F760E386EB9DE00E94470D83E511
:1050700092E00197F1F760E286EB9DE00E94470D18
:105080008091BB0D8062D9D584E08093BC0D8CE00B
:10509000D4D53CD682E08093BD0D86E0CED582E0AB
:1050A000CCD58BE39FE10197F1F7DF91CF91089584
:1050B0002F923F924F925F926F927F928F929F9228
:1050C000AF92BF92CF92DF92EF92FF920F931F9316
:1050D000CF93DF93CDB7DEB7C95DD3400FB6F89459
:1050E000DEBF0FBECDBF81E08093960A1092FF070E
:1050F0005E0127E6A21A2CEFB20A6E0137E4C31A4A
:105100003CEFD30AF9E06F2EF3E07F2E81E080932D
:10511000950A8093940AE12CF12C8091460B811121
:10512000C5C180918D0D807709F4C0C180919D0D1E
:1051300090919E0DA0919F0DB091A00D8F71992718
:10514000AA27BB27892B8A2B8B2B09F0AFC100E044
:10515000912C20909D0D30909E0D40909F0D509071
:10516000A00D60E08DE89DE00E945D15009709F4B8
:105170009DC1FC012081222309F498C12E3211F433
:1051800000E0E7CF253EE1F3338533FD2EC0B201C9
:10519000A10125E076956795579547952A95D1F712
:1051A000002359F1CA52DC4F4883C65DD340C9522F
:1051B000DC4F5883C75DD340C852DC4F6883C85D5D
:1051C000D340C752DC4F7883C95DD3400E94621E32
:1051D000CA52DC4F4881C65DD340C952DC4F58816A
:1051E000C75DD340981262C108C03F3049F626FF20
:1051F000B0CF022F0F719584ACCF21E06DE87DE038
:1052000086E49BE00E94C115882309F44FC1D501B3
:105210001C9211961C928091460B81111BC0F601C5
:1052200017C060E086E49BE00E94AA164C0100973C
:10523000E1F0FC0168E090E020E08081803209F03C
:105240007AC02F5F31962B30C1F7F601E90FF11DBF
:1052500010820BC09091490B911189C0807609F39F
:105260008FE2D6018C9311961C928091460B81FDA2
:105270005DC0982F9077C1F1DF92CF927F926F92AD
:105280003AE4832E34E0932E9F928F922AE12E9D52
:10529000C0012F9D900D1124E1E0F0E0EC0FFD1F07
:1052A0008E0F9F1F9F938F930E947642D601539635
:1052B0001C92DF92CF927F926F929F928F9224E105
:1052C0002E9DC0012F9D900D1124845C974F9F93BC
:1052D0008F930E947642BFEFEB1AFB0A0FB6F89449
:1052E000DEBF0FBECDBF22C083FF20C02AE12E9DAE
:1052F000C0012F9D900D1124B60121E030E02C0F4C
:105300003D1F820F931F0E946F42D60153961C923D
:1053100024E12E9DC0012F9D900D1124B601845CC7
:10532000974F0E946F42BFEFEB1AFB0A86E49BE0A7
:105330000E940A19F2CE283041F4A601490F511DEE
:105340003EE2DA013C939F5F60E180813FEB380FE2
:105350003A3130F4D4011C963C91362309F0805E3A
:10536000A601490F511DDA018C939F5F6ACF80918E
:105370004E0B90914F0BA091500BB091510B60913F
:105380004C0B70914D0B0097A105B10539F4C50187
:105390000E94A715882309F442CF10C020E2F5012E
:1053A00011922A95E9F720E1F501208321E022837B
:1053B00077836683848F958FA68FB78F01E0809166
:1053C000490B801708F42BCF802E912C40914A0B6B
:1053D00050914B0B4819590960E070E0E5E0440F2B
:1053E000551F661F771FEA95D1F7C5010E94CD12A0
:1053F000882309F414CF60E0C5010E945D15FC010B
:10540000892B09F40CCF83858F3009F008CF808178
:105410008F7190E08816990609F001CF21E0821A79
:1054200091084DE0489D9001499D300D1124C60121
:10543000820F931F4F0160E0D401653028F411966C
:105440004D915C9112970BC06B3028F414964D91DE
:105450005C91159704C016964D915C911797411574
:10546000510591F02B313105C8F42F5F3F4F4F3775
:10547000510508F04FE3DC014D93CD016F5FB2E0C1
:105480008B0E911C6D30C1F62B31310538F48081C3
:1054900086FF04C0D601A20FB31F1C92D6015A96F4
:1054A0001C92808186FDE1CE0F5F89CF98E0E916DE
:1054B000F10414F481E00BC0BFE0EB16F10414F426
:1054C00082E005C0E6E1EE16F104ECF483E080939F
:1054D0003B083BEE3E0DCD52DC4F3883C35DD340DD
:1054E00032EF3E0DCC52DC4F3883C45DD34039EFF0
:1054F0003E0DCB52DC4F3883C55DD3402E2C84E16A
:10550000382E01E037C04DE1E416F10414F484E0D4
:10551000DECF84E2E816F104E4F685E0D8CF88E037
:1055200093E0CFD486EA9EE0BDD484E79EE0BAD46F
:1055300089E99AE00E940908892BD1F389E99AE068
:105540000E94E707C0979093390880933808E0914C
:10555000950A8534910509F099C02091960A211188
:105560008CC02091950A3091940A231709F4A2C0A7
:105570002093940A98E0E916F10414F4122D2BC03C
:105580008091950A813031F1AFE0EA16F10434F4EC
:10559000CB52DC4F1881C55DD3401DC08230D1F0A5
:1055A000B6E1EB16F10434F4CC52DC4F1881C45D43
:1055B000D34011C0833071F0EDE1EE16F10434F404
:1055C000CD52DC4F1881C35DD34005C085EE9EE00F
:1055D00069D401C017E09E01235F3C4F2901812C53
:1055E000912C8091950A90E0019747E0489F9001A7
:1055F000499F300D1124C901880D991D389EB001B5
:10560000399E700D1124645C774FC2010E946F4275
:105610008FEF881A980A94E1490E511CA8E08A1667
:105620009104F9F6812E912C8091960A882319F025
:1056300087ED9EE016D48FE494E043D4512C852D61
:1056400090E0881599050CF06ACF452D50E060E098
:1056500070E02AE089E99AE00E94BA0985ED9EE0AF
:1056600000D48DE093E08C0F9D1FB4E15B9E800D14
:10567000911D112426D45394E2CFE23020F0E09320
:10568000940AE15014C000933A086BCF843391051B
:1056900009F067CF20913B08E21708F062CF209114
:1056A000960A222309F45DCFE093940AEF5FE0931A
:1056B000950A57CF90913A08992341F01092FF072D
:1056C00089E093E0F2D110923A0820CD90E0873043
:1056D000910508F06EC0FC0130E02150310947E02F
:1056E0008827EC57FF4F8F4F0C942642429FC001F2
:1056F000439F900D112427C0429FC001439F900DEE
:105700001124019633C0429FC001439F900D112484
:1057100002963FC0429FC001439F900D1124039603
:105720002AE1289FB001299F700D1124A1E0B0E06B
:10573000AC0FBD1F6A0F7B1F38C0429FC001439F43
:10574000900D112404962AE1289FB001299F700D25
:105750001124E1E0F0E0EC0FFD1F6E0F7F1F25C06C
:10576000429FC001439F900D112405962AE1289F76
:10577000B001299F700D112421E030E02C0F3D1F56
:10578000620F731F12C0429FC001439F900D1124EE
:1057900006962AE1289FB001299F700D112481E00F
:1057A00090E08C0F9D1F680F791F85EE97E00E9497
:1057B0006F428091E5078F3251F465EE77E08FEF0D
:1057C00097E00E945B4286EE97E06FD19FCC89E024
:1057D00093E06BD11092960AC752DC4F0FB6F89443
:1057E000DEBF0FBECDBFDF91CF911F910F91FF9014
:1057F000EF90DF90CF90BF90AF909F908F907F9071
:105800006F905F904F903F902F900895CF93DF93CC
:105810000E945C0BEB010E94770D8F3F49F00E94C4
:105820005C0B6C1B7D0B69357240A8F380E001C0F6
:1058300081E0DF91CF910895262F6091970A7091B2
:10584000980AAC0186E49BE00C9412198F929F9207
:10585000AF92BF92CF92DF92EF92FF92CF93C82F79
:1058600010926B0B81E090E0A0E0B0E080936E0BB3
:1058700090936F0BA093700BB093710B86E69BE037
:105880009093880B8093870B1092860B8FEF9FEF7E
:10589000DC018093890B90938A0BA0938B0BB093C0
:1058A0008C0BCC2331F1C53008F0DCC020E040E0A7
:1058B00050E0BA0186E89BE00E94041C009709F4BE
:1058C000D1C020E1C29F800D911D11244097FC01A1
:1058D000E254FE4F20812F7709F0C4C038968080B3
:1058E0009180A280B38081149104A104B10421F4B9
:1058F000B9C0812C912C540120E0B501A40186E8A7
:105900009BE00E94041CFC01892B09F4ABC0838539
:1059100094858115924009F0A5C08089823009F0F4
:10592000A1C0468557854115510509F49BC02585C1
:105930002093680B8FEF820F8093690B80E091E0DA
:10594000291751F031E0380F393019F480936A0B80
:1059500089C0990F832FF4CF80936A0BC688D788AC
:10596000C114D10419F0E12CF12C04C0C4A0D5A0BD
:10597000E6A0F7A0C092720BD092730BE092740B6A
:10598000F092750BD501C401840F951FA11DB11DA7
:1059900080937A0B90937B0BA0937C0BB0937D0B41
:1059A0002189328930936D0B20936C0BCC0CDD1C5C
:1059B000EE1CFF1CC80ED91EEA1EFB1EC092820BF5
:1059C000D092830BE092840BF092850B55E0220F6E
:1059D000331F5A95E1F721503E4F232F3327269549
:1059E000C20ED31EE11CF11CC092760BD092770B35
:1059F000E092780BF092790B2389348921153105D7
:105A000021F0C901A0E0B0E004C080A191A1A2A151
:105A1000B3A1B501A4014C195D096E097F09480FB6
:105A2000591F6A1F7B1F00906A0B04C0769567950B
:105A3000579547950A94D2F7DB01CA010196A11D3B
:105A4000B11D80937E0B90937F0BA093800BB0933E
:105A5000810B453F8FE058076105710528F48CE004
:105A600080936B0B80E017C0453F5F4F6105710568
:105A700010F480E10DC084A595A5A6A5B7A58093D7
:105A8000820B9093830BA093840BB093850B80E2E1
:105A900080936B0B81E0CF91FF90EF90DF90CF90E0
:105AA000BF90AF909F908F900895CF93DF93CDB725
:105AB000DEB7A0970FB6F894DEBF0FBECDBF198238
:105AC0001A82FC0120812F3271F4218121110BC037
:105AD0008DE89DE00E940A1966E67BE08DE89DE076
:105AE0000E94A71518C021E0AC016DE87DE0CE0151
:105AF00001960E941219882371F09981907751F0D4
:105B000090E2FE013196ADE8BDE001900D929A95CC
:105B1000E1F701C080E0A0960FB6F894DEBF0FBE9B
:105B2000CDBFDF91CF910895DF92EF92FF920F9357
:105B30001F93CF93DF93CDB7DEB7E3970FB6F894FB
:105B4000DEBF0FBECDBFFC017BAB6AAB19821A82F0
:105B50008081882311F080E062C090918D0D907754
:105B6000D1F37F01EAA9FBA980818F3209F054C0EB
:105B7000EAA9FBA980818F3221F43196FBABEAAB15
:105B8000F7CF6091930D7091940DCE0101960E9414
:105B9000A715882301F38E010F5F1F4F80E2D82ED7
:105BA000AE014E5C5F4FBE016F5D7F4F8AA99BA91E
:105BB0000E94441D882379F2EAA9FBA980818823E9
:105BC00019F121E0AE014F5D5F4FB801C7010E949E
:105BD000751E81110AC0AE014F5D5F4FB801C7014C
:105BE0000E94131A882309F4B6CFF701DE0111963B
:105BF0008D2D01900D928A95E1F7C7010E940A1937
:105C00008E010F5F1F4FCCCFAE014F5D5F4FB801CC
:105C1000C7010E94131A03C00DE81DE0BFCFE39631
:105C20000FB6F894DEBF0FBECDBFDF91CF911F91AD
:105C30000F91FF90EF90DF900895CF93C82F682FBA
:105C4000607F86EB9DE00E94470D80E1C89FB00118
:105C5000112486EB9DE0CF910C94470DEF92FF92BB
:105C60000F931F93CF93DF931F921F92CDB7DEB791
:105C7000877028E0829FC0011124806469837A8341
:105C8000DCDF6981E62E7A81F72E8701085F1F4FDE
:105C9000F70161917F0186EB9DE00E945D0DE016AA
:105CA000F106B1F70F900F90DF91CF911F910F91F7
:105CB000FF90EF900895CF93DF93CDB7DEB728978D
:105CC0000FB6F894DEBF0FBECDBF98E0E6EAF2E073
:105CD000DE01119601900D929A95E1F79091BE0D1B
:105CE000961710F46FEF690FFE013196E60FF11D64
:105CF000E60FF11D9081890F806828960FB6F89401
:105D0000DEBF0FBECDBFDF91CF9197CF81E095DF92
:105D10008BE39FE10197F1F70895CF93C82F682F88
:105D20008DE30E94E80A6C2F8DE20E94E80A6C2F36
:105D300085E20E94E80A6C2F8DE10E94E80A6C2F30
:105D400087E10E94E80A6C2F8FE10E94E80A6C2F1D
:105D500087E20E94E80A6C2F8FE20E94E80A6C2F0B
:105D600081E30E94E80A6C2F89E20E94E80A6C2F06
:105D700081E20E94E80A6C2F89E10E94E80A6C2FF8
:105D80008BE10E94E80A6C2F83E20E94E80A6C2FE4
:105D90008BE20E94E80A6C2F8BE3CF910C94E80A07
:105DA00080FF02C08F9A01C08F9820910B0181FF64
:105DB00002C0206101C02F7E20930B0182FF02C030
:105DC000409A01C0409883FF02C0179A01C01798FB
:105DD00084FF02C0119A01C0119885FF02C0469A43
:105DE00001C0469886FF02C0A29A01C0A2982091E5
:105DF0000B0187FF02C0246001C02B7F20930B01A1
:105E000020910B0190FF02C0216001C02E7F2093E2
:105E10000B0191FF02C0A09A01C0A09892FF02C09E
:105E2000449A01C0449893FF02C0139A01C013988A
:105E300094FF02C0159A01C0159895FF02C0429ABE
:105E400001C0429820910B0196FF02C0206401C05E
:105E50002F7B20930B0197FF02C08D9A08958D9898
:105E600008950F931F93CF93DF938C01C0E0D0E090
:105E7000F801EC0FFD1F6491662371F0E091990A1F
:105E8000F0919A0A0190F081E02D89E99AE0199544
:105E9000892B11F02196ECCFCE01DF91CF911F918C
:105EA0000F910895CF93DF93DCDFEC0166E073E0A0
:105EB00089E99AE00E942F1D8C0F9D1FDF91CF91E1
:105EC0000895CF93DF93BC0189E99AE00E942F1DCA
:105ED000EC0166E073E089E99AE00E942F1D8C0FC7
:105EE0009D1FDF91CF910895CF92DF92EF92FF92A5
:105EF0000F931F93CF93DF9377FF1DC06A017B0140
:105F0000EC016DE20E94030A8C0144275527BA0177
:105F10004C195D096E097F092AE0CE010E94BA0979
:105F2000800F911FDF91CF911F910F91FF90EF9004
:105F3000DF90CF9008952AE0DF91CF911F910F91CC
:105F4000FF90EF90DF90CF900C94BA09CF93DF933E
:105F5000CDB7DEB7ED970FB6F894DEBF0FBECDBF5D
:105F6000789484B5826084BD84B5816084BD85B534
:105F7000826085BD85B5816085BD80916E00816040
:105F800080936E00109281008091810082608093E6
:105F900081008091810081608093810080918000E8
:105FA0008160809380008091B10084608093B10013
:105FB0008091B00081608093B000809191008260F8
:105FC00080939100809191008160809391008091F5
:105FD00090008160809390008091A1008260809306
:105FE000A1008091A10081608093A1008091A00018
:105FF00081608093A00080912101826080932101C3
:106000008091210181608093210180912001816034
:106010008093200180917A00846080937A0080913F
:106020007A00826080937A0080917A008160809308
:106030007A0080917A00806880937A001092C10083
:106040000E94DB270E94DB2788E08093C10D60E07F
:1060500086EB9DE00E94E30C59DE0E942F1160E068
:1060600080E029DE64E670E080E090E00E94240B8E
:1060700060E086EB9DE00E945D0D61E086EB9DE0B7
:106080000E945D0D62E086EB9DE00E945D0D61E087
:1060900080E011DE64E670E080E090E00E94240B76
:1060A00063E086EB9DE00E945D0D64E086EB9DE081
:1060B0000E945D0D65E086EB9DE00E945D0D00E0B5
:1060C00010E06AEF70E080E090E00E94240B00FF97
:1060D0000BC068E272E083E0C1DD60E272E084E060
:1060E000BDDD68E172E00AC060E172E083E0B6DD28
:1060F00068E072E084E0B2DD60E072E085E0AEDD91
:106100008CE19BDD0F5F1F4F0D301105D1F66AEF5B
:1061100070E080E090E00E94240B60E081E0CBDD45
:1061200066E086EB9DE00E945D0D6CE271E080E030
:1061300090E00E94240B60E081E0BDDD61E086EB31
:106140009DE00E945D0D6CE271E080E090E00E94B5
:10615000240B6AEE72E088EF92E00E945211E09107
:10616000A90AF091AA0A82E08083E091A50AF09141
:10617000A60A1082E091A70AF091A80A83E0808322
:106180001092B10AE091AD0AF091AE0A86E08083E8
:10619000E091AB0AF091AC0A808180618083E0914C
:1061A000AB0AF091AC0A808188608083E091AB0AF1
:1061B000F091AC0A808180688083E091AB0AF09115
:1061C000AC0A80818F7D808389E99AE00E948508EE
:1061D0008FEE91E067DE87ED91E064DE1092B00D06
:1061E0001092AD0D1092B20D83EB9DE09093AF0D28
:1061F0008093AE0D0E945C0B8B01E090AE0DF09091
:10620000AF0D85E3D70112968C9361E00E94E80AF6
:1062100061E0F70182810E946B0AFFB6F8948091D9
:106220006106811127C0EBEAF1E08491E5E6F1E037
:106230009491E82FF0E0EE0FFF1FEA5EFE4FA5916C
:10624000B491EC91E92321F461E085E30E946B0AAB
:1062500061E085E30E94E80A8CB580618CBD8CB555
:1062600080648CBD61E084E30E94E80A61E083E31E
:106270000E94E80A809161068F5F80936106FFBEED
:10628000E091AE0DF091AF0D82E5808311828DEA31
:106290009DE00E94DF1AE091AE0DF091AF0D61E03C
:1062A00082810E946B0AEAE0FE2E8FEF0E94720D3F
:1062B000FA94F110FACFE091AE0DF091AF0D60E0DD
:1062C00082810E946B0A20E030E0A90160E08DEA43
:1062D0009DE00E944A1B813049F00E945C0B601BCC
:1062E000710B613D774078F380E25AC02AEA31E0D1
:1062F00040E050E068E08DEA9DE00E944A1B853056
:1063000011F481E00CC074E0F72E0E94770D8093A9
:10631000B10DFA94F110F9CF8A3A59F482E08093E2
:10632000B20D8091B20D823069F0C12CD12C760172
:106330000EC00E945C0B601B710B613D7740B0F298
:1063400085E22EC0C12CD12CE12C60E4F62E20E099
:1063500030E0A90167E38DEA9DE00E944A1BA70196
:10636000960169E28DEA9DE00E944A1B882349F06C
:106370000E945C0B601B710B613D774040F383E42E
:106380000FC08091B20D823001F520E030E0A9010C
:106390006AE38DEA9DE00E944A1B882341F087E36F
:1063A0008093AD0D8DEA9DE00E947E0D51C00E944C
:1063B000770D807C803C19F483E08093B20D0E94BD
:1063C000770D0E94770D0E94770D8DEA9DE00E9467
:1063D0007E0DE091AE0DF091AF0D80E5808381E000
:1063E00081838DEA9DE09093670B8093660B8DE827
:1063F0009DE00E940A1981E029DA882349F066E6C7
:106400007BE08DE89DE00E94A715882309F105C077
:1064100080E01CDA8111F3CF1BC080918D0D807755
:10642000B9F08DE89DE09093980A8093970A83ECE9
:1064300091E017DD20E030E0A90169E08DEA9DE000
:106440000E944A1B882341F083E58093AD0D48C02C
:106450008DEC91E027DD94C040E150E0BE016F5F1C
:106460007F4F8DEA9DE00E94F81A8823C9F18DEADA
:106470009DE00E947E0D8981807CB9F56F816370FB
:1064800070E0762F6627770F770F8885A4E08A9FC4
:10649000C0011124682B792B898582958695869574
:1064A0008370682B6F5F7F4FCB01A0E0B0E04A851F
:1064B0004370440F2B8527FB222720F9422B2E8186
:1064C0002F7030E0240F311D27503109BC01CD0160
:1064D00004C0660F771F881F991F2A95D2F734C012
:1064E0008DEA9DE00E947E0D2CC0803451F54A85D6
:1064F00050E060E070E04F5F5F4F6F4F7F4F8985E6
:1065000090E0A0E0B0E0BA2FA92F982F8827480F7D
:10651000591F6A1F7B1F88858F7390E0A0E0B0E051
:10652000DC0199278827840F951FA61FB71FBC0180
:10653000CD014AE0660F771F881F991F4A95D1F752
:1065400003C060E070E0CB010E94F5402FE530E72A
:1065500049E055E30E94AB4142E00E94FD2666E01F
:1065600073E089E99AE00E942F1D8CEB91E079DCC1
:1065700080916B0B90E00E94C42688E093E0A1DC40
:106580000E94E621FE0131961F0111E00FE189E929
:106590009AE00E94090820910C071816190624F4A5
:1065A000222311F40C947C3D222311F40C94783DA9
:1065B0008091EC06813409F049C08091ED06853563
:1065C00009F022C78091EE06843511F00C94473D06
:1065D0008091EF068F3411F00C94473D0E945C0BC4
:1065E0006093E8067093E9068093EA069093EB06C1
:1065F0000E94BF100E9496110E94BF100E941A268E
:106600001092FF0789E093E050DA0E9458280E9418
:106610005C0B6093E8067093E9068093EA0690931A
:10662000EB0680916006813019F40E94F624C3C6FF
:106630009EEF980F923018F40E94CB23BCC6845072
:10664000823008F0B8C60E94DD3DB5C68234E1F460
:106650008091ED06833411F00C94473D8091EE0655
:10666000863411F00C94473D0E945C0B6093E80661
:106670007093E9068093EA069093EB060E94BF10A0
:106680000E941A260C94473D853409F09DC08091E4
:10669000ED06853409F58091EE06833411F00C94F3
:1066A000473D1092E8061092E9061092EA06109211
:1066B000EB0687EA9AE0F6DB00E010E060E0C80154
:1066C0000E94933F0F5F1F4F0115F0E11F07B1F7C5
:1066D00080E99AE00C943E3D823509F04DC08091EE
:1066E000EE06863481F40E945C0B6093E80670939A
:1066F000E9068093EA069093EB060E94BF100E9481
:1067000096110C94473D823511F00C94473D0E9440
:106710005C0B6093E8067093E9068093EA06909319
:10672000EB068AEE98E0BEDB8BE093E00E949A12C3
:106730000E94220EC12CD12C7601809148029091AA
:106740004902C816D90660F44FEF5FEFC701B601E2
:106750000E94150F2FEFC21AD20AE20AF20AEDCFF9
:106760000E941F0E63E173E08EE193E00E945211DC
:1067700089ED98E00C943E3D833511F00C94473D33
:106780008091EE068F3511F00C94473D1092E8068B
:106790001092E9061092EA061092EB060091EF06BD
:1067A00010E00053110964E273E089E99AE00E9465
:1067B0000A0AC8010E94C426012B19F412980C94ED
:1067C000473D129A0C94473D823509F094C180915F
:1067D000ED06843409F09AC58091EE06813419F5EE
:1067E0008091EF06843511F00C94473D1092E80635
:1067F0001092E9061092EA061092EB0689E89AE0F8
:1068000030DB0E94250EAC0160E070E020E189E9F8
:106810009AE00E94BA0966E073E089E99AE00E9472
:106820002F1D0C94473D823509F0A2C089E79AE0FC
:1068300039DB0E945C0B6093E8067093E906809355
:10684000EA069093EB0689EC98E02CDB86E393E074
:106850000E949A1289E093E028D9CE0181960E9485
:10686000B921E1E2F0E0EC0FFD1FE80FF11D87FD1B
:10687000FA95108219821A826EE373E0C10154D92D
:106880008EE393E012D9BE016F5D7F4F85EE97E0F6
:106890000E946F4267E473E085EE97E00E945B42DE
:1068A00087EB98E0FFDA85EE97E00BDB63E485EE9B
:1068B00097E00E941C2C811103C08EE998E0BEC0B5
:1068C000C12CD12C7601BB24BA94809148029091BE
:1068D0004902A0E0B0E0C816D906EA06FB0608F0B7
:1068E00040C02601370100E010E0C301B2010E9460
:1068F000F20EF801E05AFB4FB18280830E5F1F4F0A
:106900003FEF431A530A630A730A0038110569F707
:1069100040E850E060E674E082E49BE00E94070EED
:10692000C11019C0A4E6B0E0A70196010E94BD3FC6
:1069300020914802309149022054310940E050E052
:106940000E94A13F822F0E9445126AE973E089E903
:106950009AE00E940A0A80E4C80ED11CE11CF11CD6
:10696000B4CF86E49BE00E940A1987E898E0BDC096
:10697000863411F00C94473D0E945C0B6093E8064E
:106980007093E9068093EA069093EB060E94BF108D
:1069900080904A0290904B02A0904C02B0904D0221
:1069A00086E798E07FDA86E393E00E949A1289E016
:1069B00093E07BD8CE0181960E94B921E1E2F0E01C
:1069C000EC0FFD1FE80FF11D87FDFA95108219826B
:1069D0001A8261E773E0C101A7D881E793E065D827
:1069E000BE016F5D7F4F85EE97E00E946F426AE7C0
:1069F00073E085EE97E00E945B4284E698E052DA0D
:106A000085EE97E05EDA63E485EE97E00E941C2C49
:106A1000882391F0B694A79497948794D501C401E4
:106A200080549109A109B1098BAB9CABADABBEAB56
:106A3000C12CD12C760149C08BE498E033DA6DE4A7
:106A400073E089E593E00E9452110C94473DC30125
:106A5000B2010E94320FF801E05AFB4F918380830C
:106A60000E5F1F4F9FEF491A590A690A790A0038C9
:106A7000110569F740E850E060E674E082E49BE0CD
:106A80000E94070ED701C6019F70AA27BB27892B3A
:106A90008A2B8B2BA9F4A4E6B0E0A70196010E94F3
:106AA000BD3F2BA93CA94DA95EA90E94A13F822F01
:106AB0000E9445126AE973E089E99AE00E940A0A95
:106AC000A0E4CA0ED11CE11CF11CC814D904EA04CC
:106AD000FB0428F42601370100E010E0B8CF86E47B
:106AE0009BE00E940A1983E398E0DCD963E173E03C
:106AF00086E693E0A8CF873509F0FCC08091ED06CB
:106B0000823509F0C4C78091EE06823509F0C2C013
:106B10000FEF17E01092FF0789E093E00E94552DD8
:106B20000E9458280E945C0B6093E8067093E90667
:106B30008093EA069093EB068EE793E00E949A1208
:106B400083E298E0AFD985EE97E09F938F931F93F0
:106B50000F938AE893E09F938F931F930F930E9464
:106B6000764284E198E07DD9C801ABD961E0C801E3
:106B70000E941C2C0FB6F894DEBF0FBECDBF882339
:106B800009F485C080915E0B90915F0BA091600B22
:106B9000B091610B80935C0490935D04A0935E04BC
:106BA000B0935F0440914A0250914B0260914C02B5
:106BB00070914D02481759076A077B0718F486EF52
:106BC00097E070D90E94220EC12CD12C76018090C2
:106BD000480290904902A12CB12CC814D904EA04AF
:106BE000FB0408F044C040E850E060E674E086E44E
:106BF0009BE00E94911300E614E02601370120E497
:106C00002C0DD8014C9150E05F6FC301B2012DAF44
:106C10000E94150F0E5F1F4FBFEF4B1A5B0A6B0AE6
:106C20007B0A2DAD2411EDCFD701C6018F779927AF
:106C3000AA27BB27892B8A2B8B2B99F4A4E6B0E0DB
:106C4000A70196010E94BD3FA50194010E94A13FAA
:106C5000822F0E9445126AE973E089E99AE00E9456
:106C60000A0AE0E4CE0ED11CE11CF11CB0CF89EC85
:106C700097E018D963E173E08EE793E00E94521128
:106C80000E941F0E86E49BE00E940A1900C78FED48
:106C900097E0F4C6863409F0FAC61092FF0789E03F
:106CA00093E00E94552D0E9458280E945C0B60932F
:106CB000E8067093E9068093EA069093EB068091CC
:106CC0006006813019F40E94F6240BC09EEF980FE5
:106CD000923018F40E94CB2304C08450823008F410
:106CE0006CD764E670E080E090E00E94240B0E9484
:106CF000BF1009C3803509F0EEC28091ED068235E0
:106D000009F008C48091EE06823409F0E3C0809156
:106D1000EF06823509F069C01092E8061092E90684
:106D20001092EA061092EB06809048029090490279
:106D3000A12CB12C80E993E00E949A12C12CD12C95
:106D40007601D501C40180549109A109B1098BAB29
:106D50009CABADABBEABC814D904EA04FB0408F08D
:106D6000B5C22601370100E010E0C301B2010E9464
:106D7000F20EF801EC59F94F80839FEF91830E5F7B
:106D80001F4FAFEF4A1A5A0A6A0A7A0A00381105E9
:106D900061F740E850E064E676E089E99AE00E9415
:106DA000AD07D701C6019F70AA27BB27892B8A2B65
:106DB0008B2BA9F4A4E6B0E0A70196010E94BD3F89
:106DC0002BA93CA94DA95EA90E94A13F822F0E9438
:106DD00045126AE973E089E99AE00E940A0AB0E480
:106DE000CB0ED11CE11CF11CB6CF8091EF0686348E
:106DF00009F04DC61092E8061092E9061092EA06D4
:106E00001092EB060E94BF1080904A0290904B02B5
:106E1000A0904C02B0904D0280E993E00E949A123B
:106E2000B694A79497948794D501C401805491098E
:106E3000A109B1098BAB9CABADABBEABC12CD12CC6
:106E40007601C814D904EA04FB0408F03FC2260105
:106E5000370100E010E0C301B2010E94320FF801D7
:106E6000EC59F94F808391830E5F1F4F9FEF491AB2
:106E7000590A690A790A0038110569F740E850E0B3
:106E800064E676E089E99AE00E94AD07D701C60181
:106E90009F70AA27BB27892B8A2B8B2BA9F4A4E6EA
:106EA000B0E0A70196010E94BD3F2BA93CA94DA9C6
:106EB0005EA90E94A13F822F0E9445126AE973E0F9
:106EC00089E99AE00E940A0AA0E4CA0ED11CE11CDA
:106ED000F11CB7CF843509F0DAC58091EF0686340E
:106EE00009F0FCC081E69AE00E94522F1092E80659
:106EF0001092E9061092EA061092EB060E94BF106B
:106F0000C0904A02D0904B02E0904C02F0904D02AB
:106F100080E993E00E949A1246015701B694A79423
:106F200097948794D501C4010897A109B1098FAB43
:106F300098AFA9AFBAAFC12CD12C7601C814D9042F
:106F4000EA04FB0408F0C2C1D701C601880F991FEB
:106F5000AA1FBB1FBF93AF939F938F93A5EAB3E084
:106F6000BF93AF933F922F920E947642B10189E97D
:106F70009AE00E940A0A68EE73E089E99AE00E94AA
:106F80000A0A0FB6F894DEBF0FBECDBF2601370147
:106F90009601285F3F4F3CAF2BAFC301B2010E9467
:106FA000320F9CAB8BAB99279F938F93ABEAB3E0E7
:106FB000BF93AF933F922F920E9476420F900F9013
:106FC0000F900F900F900F9000E010E0F1010190F2
:106FD0000020E9F73197E219F30982E090E08E1B77
:106FE0009F0B0817190748F468EC73E089E99AE0E9
:106FF0000E940A0A0F5F1F4FE9CFB10189E99AE0A9
:107000000E940A0A68EE73E089E99AE00E940A0A7F
:107010001F92FCA9FF93ABEAB3E0BF93AF933F92FB
:107020002F920E9476420F900F900F900F900F902A
:107030000F9000E010E0F10101900020E9F7319796
:10704000E219F30982E090E08E1B9F0B08171907E5
:1070500048F468EC73E089E99AE00E940A0A0F5F3D
:107060001F4FE9CFB10189E99AE00E940A0A68EE50
:1070700073E089E99AE00E940A0AFFEF4F1A5F0A5B
:107080006F0A7F0A2BAD3CAD2415350509F085CF7D
:1070900088E093E00E94612FD701C6019F70AA2764
:1070A000BB27892B8A2B8B2B99F4A4E6B0E0A70190
:1070B000960163D72FA938AD49AD5AAD42D7822F7B
:1070C0000E9445126AE973E089E99AE00E940A0A7F
:1070D00038E0C30ED11CE11CF11C30CF823509F021
:1070E000D6C48AE49AE00E94522F1092E8061092C9
:1070F000E9061092EA061092EB0640904802509082
:107100004902612C712C80E993E00E949A127694D6
:10711000679457944794D301C2010897A109B10914
:107120008BAB9CABADABBEABC12CD12C7601C414E8
:10713000D504E604F70408F0C9C0D701C601880FDA
:10714000991FAA1FBB1FBF93AF939F938F93A5EA6D
:10715000B3E0BF93AF933F922F920E947642B1016A
:1071600089E99AE00E940A0A68EE73E089E99AE0E8
:107170000E940A0A0FB6F894DEBF0FBECDBF4601CB
:1071800057019601285F3F4F38AF2FABC501B401BF
:107190000E94F20E99279F938F93ABEAB3E0BF93BF
:1071A000AF933F922F920E9476420F900F900F90D4
:1071B0000F900F900F9000E010E0F101019000207F
:1071C000E9F73197E219F30982E090E08E1B9F0BFB
:1071D0000817190748F468EC73E089E99AE00E94FF
:1071E0000A0A0F5F1F4FE9CFB10189E99AE00E94B7
:1071F0000A0A68EE73E089E99AE00E940A0A1F927F
:10720000FFEFFF93ABEAB3E0BF93AF933F922F92B0
:107210000E9476420F900F900F900F900F900F905A
:1072200000E010E0F10101900020E9F73197E21948
:10723000F30982E090E08E1B9F0B0817190748F4B2
:1072400068EC73E089E99AE00E940A0A0F5F1F4F19
:10725000E9CFB10189E99AE00E940A0A68EE73E079
:1072600089E99AE00E940A0AFFEF8F1A9F0AAF0A83
:10727000BF0A2FA938AD2815390509F087CF88E056
:1072800093E00E94612FD701C6018F779927AA2723
:10729000BB27892B8A2B8B2B99F4A4E6B0E0A7019E
:1072A00096016BD62BA93CA94DA95EA94AD6822F7F
:1072B0000E9445126AE973E089E99AE00E940A0A8D
:1072C00038E0C30ED11CE11CF11C31CF63E173E047
:1072D0008CE993E0B8CB8934E9F58091ED068434EC
:1072E00009F0D5C38091EE06863409F0D0C30E9420
:1072F0005C0B6093E8067093E9068093EA0690932E
:10730000EB060E94970F0E94BF10C1C3833509F09E
:1073100083C18091EE06843509F0B9C38091EF06F0
:10732000863409F0B4C30E945C0B6093E806709346
:10733000E9068093EA069093EB0688E39AE00E94C0
:10734000522F1092E8061092E9061092EA06109267
:10735000EB06D9CF8834D1F48091ED06823509F05F
:1073600096C38091EE06833509F091C38091EF06B4
:10737000843509F08CC31092E8061092E906109249
:10738000EA061092EB060C94000081C3863519F5CD
:107390008091ED068235A1F48091EE06863409F0E5
:1073A00076C30E945C0B6093E8067093E9068093B5
:1073B000EA069093EB060E94BF100E94A32267C3C7
:1073C000853409F064C38091EE06823509F05FC30D
:1073D00089E392E05AC3833509F05CC08091ED06E1
:1073E000833409F0A9C11092E8061092E9061092C0
:1073F000EA061092EB068DE19AE00E94522F0E945D
:10740000E62182E19AE03AC3843409F040C38091D6
:10741000EE06843409F03BC38091EF06823509F013
:1074200036C38091F0068F3509F031C31092E8061B
:107430001092E9061092EA061092EB066091F206AD
:107440008091F10687D3C82ED12CE12CF12CFE2C93
:10745000ED2CDC2CCC246091F4068091F3067AD3D9
:10746000C82AFE2CED2CDC2CCC246091F6068091F1
:10747000F50670D3C82A88EF99E00E94312F40E1C9
:1074800050E0C701B6010E94DA26C701B6010E948A
:10749000520EFDC2843409F0FAC28091ED068134A7
:1074A00009F0F5C28091EE06843509F0F0C28091B2
:1074B000EF06813409F0EBC28091F0068F3509F0B8
:1074C000E6C21092E8061092E9061092EA061092BF
:1074D000EB066091F2068091F1063CD3C82ED12CC8
:1074E000E12CF12CFE2CED2CDC2CCC246091F4064C
:1074F0008091F3062FD3C82A81EE99E00E94312FA4
:1075000040E150E0C701B6010E94DA26C6010E94A0
:10751000D02EBDC28D3409F0BAC21092E806109286
:10752000E9061092EA061092EB0680E897E00E94C6
:10753000522F80E697E00E94522F87E197E00E9449
:10754000522F84EE96E00E94522F80EA96E00E942D
:10755000522F8AE796E00E94522F8DE496E00E9417
:10756000522F8DE296E00E94522F8EE096E00E940C
:10757000522F87EE95E00E94522F81EC95E00E94F9
:10758000522F8DE995E00E94522F8BE695E00E94E4
:10759000522F88E395E00E94522F86E095E00E94EA
:1075A000522F84ED94E00E94522F85EA94E00E94CD
:1075B000522F86E894E00E94522F88E694E00E94C1
:1075C000522F80E494E00E94522F80E294E00E94C7
:1075D000522F8CEE93E00E94522F87EA93E00E9494
:1075E000522F83E693E00E94522F86E293E00E949E
:1075F000522F8DEE92E00E94522F83EC92E00E9477
:10760000522F83EA92E00E94522F84E892E00E9477
:10761000522F8CE392E032C2813409F0BCC08091D9
:10762000EE06843409F033C28091EF06843409F009
:107630002EC21092E8061092E9061092EA06109205
:10764000EB06C0900801C1FACC24C0F8D12CE12C83
:10765000F12CA59B02C06894C1F85A9B02C06894A3
:10766000C2F88091020180FF02C06894C3F8749B45
:1076700002C06894C4F88E9B02C06894C5F88091DB
:107680000B0181FF02C06894C6F880910B0185FF51
:1076900002C06894C7F88C9B02C06894D0F8759BB0
:1076A00002C06894D1F88091020181FF02C0689401
:1076B000D2F85B9B02C06894D3F8739B02C06894B5
:1076C000D4F88091080180FF02C06894D5F88091B9
:1076D000080182FF02C06894D6F88091080184FFF7
:1076E00002C06894D7F88091080185FF02C06894B1
:1076F000E0F8A19B02C06894E1F8419B02C0689445
:10770000E2F880910B0183FF02C06894E3F8809156
:107710000B0187FF02C06894E4F85F9B02C0689485
:10772000E5F8439B02C06894E6F88AEC99E00E9471
:10773000312F40E150E082C1843409F0A4C080912F
:10774000EE06863409F0A3C10E945C0B6093E80644
:107750007093E9068093EA069093EB060FEF17E02B
:107760001092FF0789E093E00E94552D0E9458284F
:1077700085EE97E09F938F931F930F938AE893E092
:107780009F938F931F930F93B1D60FB6F894DEBFDC
:107790000FBECDBF7CC1873409F079C18091EE0660
:1077A000883409F074C10E945C0B6093E806709302
:1077B000E9068093EA069093EB0686EB99E00E9437
:1077C000522F810150EFC52E5EEFD52EEE24EA94A4
:1077D000FE2CC701B6010E94320FD8018C9311967E
:1077E0009C93BFEFCB1ADB0AEB0AFB0A0E5F1F4F1D
:1077F000E7EFCE16EEEFDE06EFEFEE06FE0649F7F8
:107800001F868FE292E00E94312FC1010E94612FFA
:107810006CEF7EEF8FEF9FEF0E94F71088AB19AAF5
:107820001AAA82E292E00E94312FCE01C0960E94F5
:10783000612F6DEF7EEF8FEF9FEF0E94F71089A30E
:107840001AA26EEF7EEF8FEF9FEF0E94F7108BA3CF
:107850001CA21DA286E192E00E94312FCE018196EA
:107860000E94612F6FEF7EEF8FEF9FEF0E94320F2C
:10787000182F85E092E00E94312F812F110F990B74
:107880000E94C42604C1823509F073C08091EE06BF
:10789000833509F0FCC08091EF068F3509F0F7C001
:1078A0001092E8061092E9061092EA061092EB0692
:1078B00082EA99E00E94312F8091F0068093E506DC
:1078C0008091F1068093E6061092E7066EEA73E077
:1078D00089E99AE00E940A0A85EE96E0FFD2182F05
:1078E0000E94C42661E070E080E090E004C0660F72
:1078F000771F881F991F1A95D2F761157105F1E05E
:107900008F07910561F06115710524E082079105EB
:1079100031F06115710530E48307910591F48B0115
:107920009C0143E036952795179507954A95D1F721
:1079300010934902009348024AE050E00E94DA2680
:10794000A6C080E090E290934902809348022AE02A
:1079500040E050E061E070E089E99AE00E94BA09F5
:1079600066E073E089E99AE00E942F1D83E699E0C2
:1079700085C0863409F085C08091EE06833509F014
:1079800086C08091EF068F3509F081C01092E8061D
:107990001092E9061092EA061092EB068EE499E046
:1079A0000E94312F8091F0068093E5068091F106C8
:1079B0008093E6061092E7066EEA73E089E99AE0A2
:1079C0000E940A0A85EE96E089D2182F0E94C426EA
:1079D000C12CD12C7601C39404C0CC0CDD1CEE1C50
:1079E000FF1C1A95D2F74AE050E0C701B6010E9489
:1079F000DA26C114D104E10481E0F80661F0C11473
:107A0000D104E10498E0F90631F0C114D104E10495
:107A1000A0E1FA06B1F4D701C60123E0B695A79517
:107A2000979587952A95D1F780934A0290934B02B8
:107A3000A0934C02B0934D024AE050E0C701B6015A
:107A40007DCF80E090E0A0E2B0E080934A02909386
:107A50004B02A0934C02B0934D022AE040E050E06C
:107A600060E071E089E99AE00E94BA0966E073E09B
:107A700089E99AE00E942F1D8AE099E00E94522F26
:107A800006C08E3421F480E392E00E94612F809141
:107A9000E8069091E906A091EA06B091EB06892BE1
:107AA0008A2B8B2BF9F088EF98E00E94312F0E94EF
:107AB0005C0B0091E8061091E9062091EA063091EE
:107AC000EB06601B710B820B930B8FD320E030E031
:107AD0004AE754E4F6D242E00E94FD2681EB93E0AF
:107AE0000E94612F10920C071092E4061092EC068F
:107AF0000E94A6080C94C53289E99AE00E94E70723
:107B0000909163069923F1F0909162068E3381F093
:107B1000E92FF0E0E451F94F80839F5F903220F429
:107B2000909362060C94C732009362060C94C7329D
:107B3000109263069093E4061092620610930C076D
:107B40000C94C7328C3311F00C94C7321093630637
:107B50000C94C7320F931F93CF93DF931F92CDB72F
:107B6000DEB7082E000C990B698387D4182F082ED6
:107B7000000C990B77D46981892BC1F01A330CF072
:107B80001750862F660F990B78D4082F082E000CFB
:107B9000990B68D4892B51F00A330CF00750802FD1
:107BA00090E1199F800D1124805301C080E00F9057
:107BB000DF91CF911F910F9108958F929F92AF9275
:107BC000BF92CF92DF92EF92FF920F931F93CF93CA
:107BD000DF938EE793E00E949A1285EE97E09F93E1
:107BE0008F938FEF97E09F938F932AE833E03F9333
:107BF0002F939F938F937AD487E49DE00E94312F37
:107C00008FEF97E00E94612F86E39DE00E94312F65
:107C100061E08FEF97E00E941C2C2DB73EB7285FE4
:107C20003F4F0FB6F8943EBF0FBE2DBF882309F417
:107C3000E3C080915E0B90915F0BA091600BB091BF
:107C4000610B80935C0490935D04A0935E04B093F9
:107C50005F0440914A0250914B0260914C02709136
:107C60004D0284179507A607B70721F081E19DE033
:107C70000E94522F0E94220EC12CD12C7601CBE300
:107C8000D6E080915C0490915D04A0915E04B09177
:107C90005F04B695A79597958795C816D906EA0605
:107CA000FB0608F089C040E450E060E674E086E43A
:107CB0009BE00E9491134AEA50E065E575E080E0A0
:107CC00090E00E94700F45E550E06AEA72E080E0C3
:107CD00090E00E94700F45E250E0C701B6010E949B
:107CE000700F4FE150E0C701B6010E94700F409144
:107CF000610450E0542F442780916004482BC70151
:107D0000B6010E94700F460157013FEF831A930A94
:107D1000A30AB30A02E010E0F801E05AFB4F4181E8
:107D200050E0542F44278081482BC501B4010E94A4
:107D3000700F0E5F1F4F8FEF881A980AA80AB80AB3
:107D40000034110549F749E250E0C701B6010E942D
:107D5000700FCE010197F1F7D701C6019F70AA27D6
:107D6000BB27892B8A2B8B2B09F5A4E6B0E0A70152
:107D7000960103D100915C0410915D0420915E0492
:107D800030915F043695279517950795A9019801BD
:107D90002052310941095109D4D0822F0E94451245
:107DA0006AE973E089E99AE00E940A0A20E2C20EB9
:107DB000D11CE11CF11C65CF88E093E00E94612F8B
:107DC00083EE9CE00E94522F63E173E08EE793E024
:107DD0000E9452110E941F0E86E49BE0DF91CF911A
:107DE0001F910F91FF90EF90DF90CF90BF90AF90D9
:107DF0009F908F900C940A198AEF9CE0DF91CF91AD
:107E00001F910F91FF90EF90DF90CF90BF90AF90B8
:107E10009F908F900C94522FE9E9FAE0138212821E
:107E200088EE93E0A0E0B0E084839583A683B783D7
:107E300022EB32E03183208325EC30E03587248744
:107E400024EC30E03787268720EC30E0318B208B24
:107E500021EC30E0338B228B22EC30E0358B248B0D
:107E600026EC30E0378B268B118E128E138E148EFB
:107E7000E6E3FBE01382128284839583A683B783B3
:107E800084EC92E091838083E6EBFDE01382128222
:107E900082EE92E09183808387E2848380E1818710
:107EA00082E08287138610926B0B10928D0D1092D8
:107EB0008E0D84E68093AD0D1092B20D80E5809317
:107EC000B30D1092B40DE2E4FBE01482158213822C
:107ED000128286ED92E0918380830895FC018827C9
:107EE0009927E89421912032E9F3293010F02E30BF
:107EF000C8F32B3239F02D3231F4689403C00BD023
:107F0000820F911D219120532A30C8F31EF49095C1
:107F100081959F4F08957AE0979F902D879F802DA0
:107F2000910D11240895262FF999FECF1FBA92BD05
:107F300081BD20BD0FB6F894FA9AF99A0FBE01964A
:107F40000895052E97FB16F400940FD057FD05D029
:107F50001ED007FC02D046F408C0509540953095DD
:107F600021953F4F4F4F5F4F0895909580957095A5
:107F700061957F4F8F4F9F4F08952BD0A59F900DF8
:107F8000B49F900DA49F800D911D11240895A1E22E
:107F90001A2EAA1BBB1BFD010DC0AA1FBB1FEE1F83
:107FA000FF1FA217B307E407F50720F0A21BB30BCE
:107FB000E40BF50B661F771F881F991F1A9469F74A
:107FC00060957095809590959B01AC01BD01CF01A6
:107FD0000895A29FB001B39FC001A39F700D811DA2
:107FE0001124911DB29F700D811D1124911D0895C2
:107FF0005058BB27AA270ED070C161D130F066D18E
:1080000020F031F49F3F11F41EF456C10EF4E095B8
:10801000E7FB4CC1E92F72D180F3BA1762077307EF
:108020008407950718F071F49EF58AC10EF4E09567
:108030000B2EBA2FA02D0B01B90190010C01CA0122
:10804000A0011124FF27591B99F0593F50F4503ECD
:1080500068F11A16F040A22F232F342F4427585FBF
:10806000F3CF469537952795A795F0405395C9F7D7
:108070007EF41F16BA0B620B730B840BBAF091508F
:10808000A1F0FF0FBB1F661F771F881FC2F70EC02E
:10809000BA0F621F731F841F48F487957795679501
:1080A000B795F7959E3F08F0B3CF9395880F08F0EA
:1080B0009927EE0F979587950895D4D008F481E01D
:1080C00008950CD00AC102D140F0F9D030F021F46B
:1080D0005F3F19F0EBC0511134C1EEC00FD198F3DE
:1080E0009923C9F35523B1F3951B550BBB27AA2739
:1080F00062177307840738F09F5F5F4F220F331FAB
:10810000441FAA1FA9F333D00E2E3AF0E0E830D076
:1081100091505040E695001CCAF729D0FE2F27D079
:10812000660F771F881FBB1F261737074807AB0747
:10813000B0E809F0BB0B802DBF01FF2793585F4FBC
:108140002AF09E3F510568F0B1C0FBC05F3FECF3E1
:10815000983EDCF3869577956795B795F7959F5F81
:10816000C9F7880F911D9695879597F90895E1E0D5
:10817000660F771F881FBB1F621773078407BA0734
:1081800020F0621B730B840BBA0BEE1F88F7E0958F
:108190000895BCD088F09F5790F0B92F9927B75118
:1081A000A0F0D1F0660F771F881F991F1AF0BA95BB
:1081B000C9F712C0B13081F0C3D0B1E00895C0C09A
:1081C000672F782F8827B85F39F0B93FCCF38695B1
:1081D00077956795B395D9F73EF49095809570950E
:1081E00061957F4F8F4F9F4F0895E89409C097FB8B
:1081F0003EF490958095709561957F4F8F4F9F4F7E
:108200009923A9F0F92F96E9BB279395F6958795C1
:1082100077956795B795F111F8CFFAF4BB0F11F484
:1082200060FF1BC06F5F7F4F8F4F9F4F16C088232B
:1082300011F096E911C0772321F09EE8872F762F61
:1082400005C0662371F096E8862F70E060E02AF0A2
:108250009A95660F771F881FDAF7880F969587958E
:1082600097F90895990F0008550FAA0BE0E8FEEF63
:1082700016161706E807F907C0F012161306E407EA
:10828000F50798F0621B730B840B950B39F40A26E3
:1082900061F0232B242B252B21F408950A2609F4C1
:1082A000A140A6958FEF811D811D089597F99F67C5
:1082B00080E870E060E008959FEF80EC089500246E
:1082C0000A941616170618060906089500240A943B
:1082D00012161306140605060895092E0394000CC1
:1082E00011F4882352F0BB0F40F4BF2B11F460FF50
:1082F00004C06F5F7F4F8F4F9F4F089557FD905879
:10830000440F551F59F05F3F71F04795880F97FB59
:10831000991F61F09F3F79F0879508951216130613
:108320001406551FF2CF4695F1DF08C01616170642
:108330001806991FF1CF8695710561050894089577
:10834000E894BB2766277727CB0197F908958ADF42
:1083500008F48FEF08950BD0C0CFB1DF28F0B6DF5F
:1083600018F0952309F0A2CFA7CF1124EACFC6DFDA
:10837000A0F3959FD1F3950F50E0551F629FF00138
:10838000729FBB27F00DB11D639FAA27F00DB11D91
:10839000AA1F649F6627B00DA11D661F829F22271A
:1083A000B00DA11D621F739FB00DA11D621F839FA1
:1083B000A00D611D221F749F3327A00D611D231F77
:1083C000849F600D211D822F762F6A2F11249F57C5
:1083D00050408AF0E1F088234AF0EE0FFF1FBB1FE8
:1083E000661F771F881F91505040A9F79E3F510587
:1083F00070F05CCFA6CF5F3FECF3983EDCF3869540
:1084000077956795B795F795E7959F5FC1F7FE2B31
:10841000880F911D9695879597F9089523DF880B0E
:10842000990B0895AA1BBB1B51E107C0AA1FBB1FD4
:10843000A617B70710F0A61BB70B881F991F5A95F0
:10844000A9F780959095BC01CD010895EE0FFF1F0F
:10845000881F8BBF0790F691E02D199481E090E082
:10846000F89410C391115FC280538A5028F0865C43
:10847000806281568650B8F708959111089581560B
:108480008A5108F4805285580895FB01DC0104C02C
:108490008D910190801921F441505040C8F7881BFC
:1084A000990B0895FB01DC0102C001900D9241502F
:1084B0005040D8F70895FB01DC010D900020E9F74A
:1084C000119701900D920020E1F70895FB01DC0166
:1084D0008D91019080190110D9F3990B0895FB013A
:1084E000DC0101900D920020E1F708950F931F9396
:1084F000CF93DF93CDB7DEB72E970FB6F894DEBFDC
:108500000FBECDBF0E891F8986E08C831A83098335
:108510008FEF9FE79E838D83AE01465E5F4F688D30
:10852000798DCE01019611D02F813885F801E20FA7
:10853000F31F10822E960FB6F894DEBF0FBECDBF8C
:10854000DF91CF911F910F9108952F923F924F92FB
:108550005F926F927F928F929F92AF92BF92CF92D3
:10856000DF92EF92FF920F931F93CF93DF93CDB7DC
:10857000DEB72C970FB6F894DEBF0FBECDBF7C01DF
:108580006B018A01FC0117821682838181FFB0C1D1
:10859000CE0101964C01F7019381F60193FD85917F
:1085A00093FF81916F01882309F49EC1853239F4CC
:1085B00093FD859193FF81916F01853221F4B7017D
:1085C00090E0CAD1E8CF512C312C20E02032A0F429
:1085D0008B3269F030F4803259F0833269F42061D3
:1085E0002CC08D3239F0803339F4216026C02260EE
:1085F000246023C0286021C027FD27C030ED380F3C
:108600003A3078F426FF06C0FAE05F9E300D112460
:10861000532E13C08AE0389E300D1124332E206271
:108620000CC08E3221F426FD5FC1206406C08C365A
:1086300011F4206802C0883641F4F60193FD85915B
:1086400093FF81916F018111C1CF982F9F7D955428
:10865000933028F40C5F1F4FFFE3F9830DC083367E
:1086600031F0833771F0833509F057C021C0F8012C
:10867000808189830E5F1F4F44244394512C540101
:1086800014C03801F2E06F0E711CF801A080B180B7
:1086900026FF03C0652D70E002C06FEF7FEFC501BC
:1086A0002C874FD12C0183012C852F77222E16C0C9
:1086B0003801F2E06F0E711CF801A080B18026FF36
:1086C00003C0652D70E002C06FEF7FEFC5012C87FE
:1086D0002DD12C012C852068222E830123FC19C06A
:1086E000832D90E048165906A0F4B70180E290E08F
:1086F00033D13A94F5CFF50127FC859127FE81917E
:108700005F01B70190E028D131103A94F1E04F1A9F
:1087100051084114510479F7DEC0843611F08936CE
:1087200031F5F80127FF07C0608171818281938153
:108730000C5F1F4F08C060817181072E000C880BF1
:10874000990B0E5F1F4F2F76722E97FF09C09095E1
:108750008095709561957F4F8F4F9F4F2068722E47
:108760002AE030E0A40130D1A82EA81843C08537F4
:1087700029F42F7EB22E2AE030E025C0F22FF97FB7
:10878000BF2E8F36C1F018F4883579F0ADC0803730
:1087900019F0883721F0A8C02F2F2061B22EB4FE27
:1087A0000DC08B2D8460B82E09C024FF0AC09F2FF6
:1087B0009660B92E06C028E030E005C020E130E028
:1087C00002C020E132E0F801B7FE07C0608171818C
:1087D000828193810C5F1F4F06C06081718180E0B0
:1087E00090E00E5F1F4FA401EFD0A82EA818FB2D1C
:1087F000FF777F2E76FE0BC0372D3E7FA51450F4F9
:1088000074FE0AC072FC08C0372D3E7E05C0BA2C2B
:10881000372D03C0BA2C01C0B52C34FF0DC0FE01AA
:10882000EA0DF11D8081803311F4397E09C032FFD9
:1088300006C0B394B39404C0832F867809F0B39430
:1088400033FD12C030FF06C05A2CB31418F4530C79
:108850005B18B32CB31460F4B70180E290E03C875E
:108860007BD0B3943C85F6CFB31410F43B1801C011
:10887000312C34FF11C0B70180E390E03C876CD00D
:108880003C8532FF16C031FD03C088E790E002C08E
:1088900088E590E0B7010CC0832F867851F031FF56
:1088A00002C08BE201C080E237FD8DE2B70190E0AB
:1088B00053D0A51430F4B70180E390E04DD05A9422
:1088C000F8CFAA94F401EA0DF11D8081B70190E080
:1088D00043D0A110F6CF332009F45DCEB70180E27A
:1088E00090E03AD03A94F7CFF7018681978102C0A1
:1088F0008FEF9FEF2C960FB6F894DEBF0FBECDBF63
:10890000DF91CF911F910F91FF90EF90DF90CF906B
:10891000BF90AF909F908F907F906F905F904F909F
:108920003F902F900895992788270895FC0105907E
:10893000615070400110D8F7809590958E0F9F1F61
:108940000895FC016150704001900110D8F78095A6
:1089500090958E0F9F1F08950F931F93CF93DF93D2
:10896000FB01238121FD03C08FEF9FEF28C022FF71
:1089700016C046815781248135814217530744F43C
:10898000A081B1819D012F5F3F4F318320838C9364
:10899000268137812F5F3F4F3783268310C0EB013D
:1089A000092F182F0084F185E02D1995892BE1F608
:1089B0008E819F8101969F838E83812F902FDF91DF
:1089C000CF911F910F910895FA01AA27283051F1F4
:1089D000203181F1E8946F936E7F6E5F7F4F8F4FF0
:1089E0009F4FAF4FB1E03ED0B4E03CD0670F781F4F
:1089F000891F9A1FA11D680F791F8A1F911DA11D34
:108A00006A0F711D811D911DA11D20D009F468946C
:108A10003F912AE0269F11243019305D3193DEF614
:108A2000CF010895462F4770405D4193B3E00FD0CA
:108A3000C9F7F6CF462F4F70405D4A3318F0495DB5
:108A400031FD4052419302D0A9F7EACFB4E0A69598
:108A50009795879577956795BA95C9F700976105BA
:108A6000710508959B01AC010A2E06945795479510
:108A700037952795BA95C9F7620F731F841F951F05
:088A8000A01D0895F894FFCF3A
:108A88000000000000101E000C121201010000007E
:108A98000000000102040F000000000000001C009C
:108AA8000C12121101011100000000000102070060
:108AB800556E6974202331370056425F50524F4734
:108AC80020312E30000000000020000020001E038E
:108AD800191D1D19031E1E0301010101031E1F009C
:108AE8001B1B1B1B001F1F0018181818001F1F0036
:108AF80000000000001F0F1813171713180F0F1886
:108B080010101010180F1F00000000001F0E1C028C
:108B18000202021E00001F001B1B00001F0E070898
:108B28000808080F0000000040001400540000006E
:108B380000003F08AD07D80785080908E707FB07C5
:108B4800000000008A095B09040E3509530944092D
:108B58003609000000000A0E070E040E1C0E000065
:108B680000005D0DAD07040E030E50726F67726151
:108B78006D6D657220202000564220436172747228
:108B88006964676520000D0A002F004572617369EA
:108B98006E6700436F6D706C657465642100457283
:108BA8006173650053657474696E67204553206C62
:108BB800696E653A200052656164696E67005241CA
:108BC8004D5F52454144002E7372616D0066696CB9
:108BD80065206F6E205344210043616E2774206323
:108BE8007265617465005265616420746F20534436
:108BF80000524F4D5F52454144002E76620050723C
:108C08006F6772616D6D696E670025732F2573003C
:108C18005072696E74696E672E2E2E005072696EDE
:108C280074696E67002530386C7800257800325EEC
:108C380000736563730025303458003030433200C8
:108C4800303046310030303230003232323100328A
:108C580032323200303030310045726173696E67EC
:108C680020202020202020202000506C6561736582
:108C78002057616974202020202000250056657245
:108C8800696679696E67004641494C45442100563A
:108C980065726669636174696F6E0050415353452C
:108CA8004421004552524F522100534420436172DF
:108CB8006400426C616E6B20436865636B006E6193
:108CC8006E00696E66006F76660025732573005323
:0C8CD800656C6563742066696C650000C3
:00000001FF
